:100000000C94E0010C94EC330C9419340C94080219
:100010000C9408020C9408020C9408020C94080238
:100020000C9408020C9408020C9408020C94F30639
:100030000C9408020C9408020C9408020C94080218
:100040000C94F8320C9408020C9469060C94A506E2
:100050000C9408020C9408020C9408020C940802F8
:100060000C9408020C940802084AD73B3BCE016E60
:1000700084BCBFFDC12F3D6C74319ABD56833DDAFF
:100080003D00C77F11BED9E4BB4C3E916BAAAABE0E
:10009000000000803F05A84CCDB2D44EB93836A937
:1000A000020C50B9918688083CA6AAAA2ABE000074
:1000B00000803F0664EC1B3C04BC163E3BE5B93CAB
:1000C000C93C37C29E5A3D660498083EEA69AAAA0E
:1000D0003E000000803F2020BF0020BF00BF007C0A
:1000E0002020202020202020202020202020202010
:1000F00020202000C8202020202020202020202078
:1001000020C900C8202020202020202020202020BE
:10011000C97C00D820202020202020202020202042
:10012000D97C00C820202020202020202020202032
:10013000C97C00C820202020202020202020202032
:10014000C97C00206172737369006D696E6F706F96
:100150007364206C6962726570696C6F7400202032
:10016000202020BABBBCBDBE7C2020202020CACBD2
:10017000CCCDCE7C00626F6F74696E672075703A6B
:10018000EDF2F2F2F2F2F2F2F30063616C69627284
:100190006174657C7C6D6561737572656420616DE9
:1001A000703A20200063616C6962726174657C7CC6
:1001B0006D6561737572656420616D703A20200011
:1001C00063616C6962726174657C7C6D6561737575
:1001D00072656420766F6C743A2000626174746595
:1001E0007279207761726E696E6720007478706929
:1001F000642076616C756573006261726F2074654E
:100200006D700074656D7064697370200061637453
:100210006976652000706173736976650075617633
:1002200074616C6B20007365747570207363726504
:10023000656E7C7C7C004368617220446F6E650A49
:1002400000526561647920666F7220466F6E740A91
:100250000055706461746520436861725365740071
:1002600000407A10F35A00A0724E18090010A5D46D
:10027000E80000E87648170000E40B54020000CACA
:100280009A3B000000E1F505000080969800000010
:1002900040420F000000A08601000000102700006F
:1002A0000000E803000000006400000000000A00F5
:1002B000000000000100000000002C76D888DC67F8
:1002C0004F0823DFC1DFAE59E1B1B796E5E3E45350
:1002D000C63AE651997696E8E6C28426EB898C9B6D
:1002E00062ED407C6FFCEFBC9C9F40F2BAA56FA50D
:1002F000F490055A2AF75C936B6CF9676DC11BFC8F
:10030000E0E40D47FEF520E6B500D0ED902E0300A9
:10031000943577050080841E080000204E0A0000F6
:1003200000C80C333333330F986E12831141EF8DB5
:100330002114893BE65516CFFEE6DB18D1844B38F5
:100340001BF77C1D901DA4BBE424203284725E2226
:100350008100C9F124ECA1E53D276E616E00696E54
:10036000660000000000240027002A0000000000B2
:10037000250028002B000000000023002600290093
:10038000040404040404040402020202020203033B
:100390000303030301020408102040800102040843
:1003A00010200102040810200000000700020100D4
:1003B00000030406000000000000000074043A0876
:1003C00011241FBECFEFD8E0DEBFCDBF13E0A0E009
:1003D000B1E0EAECF2E702C005900D92A03FB10750
:1003E000D9F716E0A0EFB3E001C01D92A33AB10720
:1003F000E1F713E0C0ECD3E004C02297FE010E94B5
:100400005F39CC3BD107C9F70E9428350C9463397A
:100410000C940000FA01AA27283051F1203181F113
:10042000E8946F936E7F6E5F7F4F8F4F9F4FAF4FFC
:10043000B1E03ED0B4E03CD0670F781F891F9A1F0F
:10044000A11D680F791F8A1F911DA11D6A0F711DC3
:10045000811D911DA11D20D009F468943F912AE0CF
:10046000269F11243019305D3193DEF6CF010895B7
:10047000462F4770405D4193B3E00FD0C9F7F6CFE8
:10048000462F4F70405D4A3318F0495D31FD4052B0
:10049000419302D0A9F7EACFB4E0A6959795879546
:1004A00077956795BA95C9F7009761057105089525
:1004B0009B01AC010A2E06945795479537952795D1
:1004C000BA95C9F7620F731F841F951FA01D089569
:1004D000283008F027E03327DA01990F311D87FD16
:1004E000916000966105710539F432602E5F3D938D
:1004F00030E32A95E1F708959F3F30F08038710589
:10050000610509F03C5F3C5F3D93913008F08068E5
:10051000911DDF93CF931F930F93FF92EF92192FAB
:10052000987F9695E92F96959695E90FFF27E654C3
:10053000FD4F99273327EE24FF24A701E7010590FB
:100540000894079428F4360FE71EF81E491F511D22
:10055000660F771F881F991F0694A1F705900794CF
:1005600028F4E70EF81E491F561FC11D770F881F7C
:10057000991F661F0694A1F70590079428F4F80EBA
:10058000491F561FC71FD11D880F991F661F771F50
:100590000694A1F70590079420F4490F561FC71F32
:1005A000D81F990F661F771F881F0694A9F784919B
:1005B0001095177041F0D695C79557954795F794C4
:1005C000E7941A95C1F7E0E6F2E06894159015916A
:1005D00035916591959105907FE27395E118F10A47
:1005E000430B560BC90BD009C0F7E10CF11E431F9A
:1005F000561FC91FD01D7EF4703311F48A95E6CFC3
:10060000E894015030F0080F0AF40027021708F4AC
:10061000202F2395022F7A3328F079E37D932A95B2
:10062000E9F710C07D932A9589F60694979567950A
:10063000379517951794E118F10A430B560BC90B20
:10064000D00998F023957E9173957A3308F070E382
:100650007C932013B8F77E9170617D9330F0839581
:1006600071E37D9370E32A95E1F71124EF90FF90F9
:100670000F911F91CF91DF91992787FD9095089554
:10068000CF93DF93BC018230910510F462E070E0FB
:10069000A091A106B091A206ED0140E050E0E0E09B
:1006A000F0E021C0888199818617970769F48A81D3
:1006B0009B81309719F09383828304C09093A206A4
:1006C0008093A106FE0134C06817790738F44115FC
:1006D000510519F08417950708F4AC01FE018A81D1
:1006E0009B819C01E9012097E9F641155105A9F18B
:1006F000CA01861B970B049708F4BA01E0E0F0E00A
:100700002AC08D919C91119784179507F9F464176D
:10071000750781F412968D919C911397309719F07B
:100720009383828304C09093A2068093A106FD0167
:1007300032964CC0CA01861B970BFD01E80FF91FCA
:100740006193719302978D939C9340C0FD018281C8
:1007500093819C01D9011097A1F680919F069091F9
:10076000A006892B41F480918C0290918D02909388
:10077000A00680939F0640918E0250918F024115F2
:10078000510541F44DB75EB780918A0290918B027A
:10079000481B590B20919F063091A006CA01821B6D
:1007A000930B8617970780F0AB014E5F5F4F84175E
:1007B000950750F0420F531F5093A00640939F0699
:1007C000F9016193719302C0E0E0F0E0CF01DF91A5
:1007D000CF910895CF93DF93009709F450C0EC01B7
:1007E00022971B821A82A091A106B091A2061097AF
:1007F00009F140E050E0AC17BD0708F1BB83AA83C4
:10080000FE0121913191E20FF31FAE17BF0779F47A
:100810008D919C911197280F391F2E5F3F4F39837F
:10082000288312968D919C9113979B838A834115FF
:10083000510571F4D093A206C093A10620C0129670
:100840008D919C911397AD01009711F0DC01D3CFEE
:10085000FA01D383C28321913191E20FF31FCE17A6
:10086000DF0769F488819981280F391F2E5F3F4F78
:10087000FA01318320838A819B8193838283DF9174
:10088000CF910895FC010590615070400110D8F798
:10089000809590958E0F9F1F0895FC0161507040C8
:1008A00001900110D8F7809590958E0F9F1F0895A5
:1008B0006EBD0DB407FEFDCF8EB508958DE061E0ED
:1008C0000E9446348BE061E00E9446348CE060E098
:1008D0000E9446348AE061E00E9446341CBC80E5F8
:1008E0008CBD8DB58EB5089580EF93E00E945E04B7
:1008F0000895FC011382128288EE93E0A0E0B0E03C
:1009000084839583A683B78385EA92E0918380836D
:100910000895FC018089803419F421E030E002C0A0
:1009200020E030E0C9010895FC01818990E008953C
:10093000FC016487458766874787089580E090E0DB
:10094000089580E090E0089580E090E00895089593
:10095000EF92FF921F93CF93DF93162F7A0186E0D9
:1009600060E00E94853480EF93E060E00E945804CC
:1009700080EF93E060E00E94580480EF93E069E02C
:100980000E94580480EF93E0612F0E945804C0E059
:10099000D0E0F701EC0FFD1F108180EF93E06AE0DB
:1009A0000E94580480EF93E06C2F0E94580480EF5F
:1009B00093E06BE00E94580480EF93E0612F0E9467
:1009C00058042196C633D10521F780EF93E068E003
:1009D0000E94580480EF93E060EA0E94580480EF80
:1009E00093E060EA0E94580485FDF9CF80EF93E020
:1009F00060E00E94580480EF93E06CE00E9458048D
:100A000086E061E00E948534DF91CF911F91FF90D5
:100A1000EF9008951F93CF93DF93EC01162F86E09C
:100A200060E00E94853480EF93E060E00E9458040B
:100A3000112319F0113059F404C080EF93E0688954
:100A400004C068896C6180EF93E00E94580486E0DE
:100A500061E00E948534DF91CF911F910895EF925C
:100A6000FF920F931F938EE1489F70011124E60EB1
:100A7000F11C86E060E00E94853400EF13E0C801BD
:100A800065E00E945804C8016F2D0E945804C801F7
:100A900066E00E945804C8016E2D0E9458041F9100
:100AA0000F91FF90EF900895EF92FF920F931F9395
:100AB0007C0100EF13E0C80167E00E945804C80100
:100AC0006FEF0E94580486E061E00E948534F701D0
:100AD00087858F5F87871F910F91FF90EF90089513
:100AE000EF92FF920F931F93FC01E7848EE1E89E43
:100AF000700111248685E80EF11C86E060E00E94FA
:100B0000853400EF13E0C80164E00E945804C80176
:100B100063E00E945804C80165E00E945804C801BF
:100B20006F2D0E945804C80166E00E945804C80155
:100B30006E2D0E9458041F910F91FF90EF90089521
:100B40001F93CF93DF93EC01162F6C3731F40E9483
:100B50005405CE010E9470050AC080EF93E067E063
:100B60000E94580480EF93E0612F0E94580481E0B6
:100B700090E0DF91CF911F9108950F931F9386E02E
:100B800060E00E94853400EF13E0C80164E00E9439
:100B90005804C80164E00E94580486E061E00E94A5
:100BA00085341F910F9108951F93CF93DF93EC012C
:100BB000188A16E0198B8FE896E060E973E00E94CE
:100BC0005832813049F480E4888B88E0898B86E054
:100BD00060E00E94853402C0188A198B86E060E0CC
:100BE0000E948534DF91CF911F9108950F931F9339
:100BF000CF93DF93EC0186E061E00E94463482E00F
:100C000060E00E94463482E061E00E948534CE01BB
:100C10000E94D40586E060E00E94853480EF93E076
:100C20006CEE0E94580480EF93E06FEF0E9458042E
:100C3000182F80EF93E060E00E945804688962609A
:100C400080EF93E00E94580462E370E080E090E05F
:100C50000E944E3380EF93E06CE60E9458041F7EA2
:100C600080EF93E0612F0E9458048889803419F046
:100C70000DE010E002C000E110E01092F2031092CB
:100C8000F10317C06091F1037091F203605F80EF90
:100C900093E00E94580480EF93E069E00E945804BA
:100CA0008091F1039091F20301969093F203809367
:100CB000F1038091F1039091F2038017910714F3EF
:100CC000CE0161E00E940A05DF91CF911F910F9143
:100CD00008951F920F920FB60F9211242F933F93F6
:100CE0004F938F939F93EF93FF934091C600209172
:100CF0007E0630917F062F5F3F4F80918206909154
:100D00008306282339238091800690918106281735
:100D1000390779F080917E0690917F06E0918406F4
:100D2000F0918506E80FF91F408330937F062093EA
:100D30007E06FF91EF919F918F914F913F912F915F
:100D40000F900FBE0F901F9018951F920F920FB625
:100D50000F9211242F933F938F939F93EF93FF93C1
:100D600020918806309189068091860690918706A9
:100D700028173907E9F08091880690918906E0915B
:100D80008C06F0918D06E80FF91F80818093C600D4
:100D90008091880690918906019620918A0630916B
:100DA0008B0682239323909389068093880610C034
:100DB0002091860630918706809188069091890659
:100DC0002817390729F48091C1008F7D8093C100D5
:100DD000FF91EF919F918F913F912F910F900FBEB7
:100DE0000F901F9018951F920F920FB60F9211241B
:100DF0008F939F938091B3049091B404892B51F009
:100E00008091B5049091B60401969093B6048093B6
:100E1000B50409C08091B7049091B80401969093ED
:100E2000B8048093B7049F918F910F900FBE0F90DD
:100E30001F901895CF93DF93482FEB018091000608
:100E4000833009F45DC0843028F48130C1F08230F1
:100E500058F50AC0853009F4D2C0853008F4A8C01E
:100E6000863009F0F2C0E9C04C3309F0EEC081E0F1
:100E700080930006488384EB8093FF05E6C0842FAF
:100E800090E0E091FF05F0E0E827F927ED54FD4FF1
:100E900020812093FF05887F9070809741F582E044
:100EA00080930006498329C0242F30E0E091FF059C
:100EB000F0E0E227F327ED54FD4F80818093FF059A
:100EC0008091FE058F5F8093FE05823018F43B838E
:100ED0002A83BBC0922F88272A813B81820F931FD0
:100EE0009B838A830A978F3F910521F018F0109217
:100EF0000006ABC083E0809300061092FE05A5C0FB
:100F0000E42FF0E08091FF0590E0E827F927ED5409
:100F1000FD4F80818093FF056091FE056F5F6093B8
:100F2000FE05623089F0633020F4613009F08DC035
:100F300006C0633091F0643009F087C022C0842F6E
:100F400090E0A0E0B0E018C0242F30E040E050E096
:100F5000542F432F322F222707C0242F30E040E0A8
:100F600050E0A901332722278C819D81AE81BF816A
:100F7000820F931FA41FB51F8C839D83AE83BF83F5
:100F800064C0242F30E040E050E0522F4427332744
:100F900022278C819D81AE81BF81820F931FA41F68
:100FA000B51F8C839D83AE83BF8360930006A5CF5E
:100FB000242F30E0E091FF05F0E0E227F327ED5425
:100FC000FD4F80818093FF058091FE058F5F8093A8
:100FD000FE05813019F08230C1F503C039872887BA
:100FE00034C0922F882728853985280F391F3987E3
:100FF00028878A819B810A97F1F085E07CCFE42FD6
:10100000F0E08091FF0590E0E827F927ED54FD4FCF
:1010100080818093FF052091FE052F5F2093FE05C0
:1010200030E0FB01E20FF31F41878A819B810A9721
:101030002817390750F086E05ECFC75FDE4F488340
:10104000C950D14087E08093000680910006873028
:1010500069F410920006C75FDE4F9091FF0588810A
:10106000C950D140981711F48A8101C080E0DF9106
:10107000CF9108958F92AF92CF92EF92FF920F93FC
:101080001F9389E794E060E045EC50E024EC30E009
:1010900000EC10E0B1ECEB2EF12CCC24C394A8E9C9
:1010A000AA2EF0E28F2E0E94C82B86E994E00E94BF
:1010B00079041092A9041092AA041092AB04109221
:1010C000AC041092AD041092AE041092AF041092D2
:1010D000B0041092B2041092B1041092A8041F91AF
:1010E0000F91FF90EF90CF90AF908F900895AF92B7
:1010F000BF92CF92DF92EF92FF920F931F93E090F7
:101100007A06F0907B0600917C0610917D068FE5B3
:1011100090E0A0E0B0E0E80EF91E0A1F1B1F0E943D
:1011200040336E157F058007910708F44EC0A090EC
:10113000DE04B090DF04C090E004D090E104C6016A
:10114000B50120E030E040E85FE30E94C8371816A0
:1011500094F5E0902606F09027060091280610915D
:1011600029060E94403320917A0630917B064091F7
:101170007C0650917D06621B730B840B950B0E94BD
:101180009E369B01AC01C601B5010E94D33720E019
:1011900030E04AE754E40E9405369B01AC01C801E7
:1011A000B7010E9438356093260670932706809316
:1011B0002806909329060E94403360937A06709324
:1011C0007B0680937C0690937D061F910F91FF9084
:1011D000EF90DF90CF90BF90AF900895AF92BF9205
:1011E000DF92EF92FF920F931F93CF93DF938C01C7
:1011F0008091010680FDE4C0F801F08089E794E069
:101200006F2D0E94A92CE801C75FDE4FEF2DF0E0A3
:10121000ED54FD4F80818883F801F18089E794E0E7
:101220006F2D0E94A92CEF2DF0E0888190E0E82737
:10123000F927ED54FD4F80818883F801F28089E71A
:1012400094E06F2D0E94A92CEF2DF0E0888190E0B2
:10125000E827F927ED54FD4F80818883F801F3805A
:1012600089E794E06F2D0E94A92CEF2DF0E0888192
:1012700090E0E827F927ED54FD4F80818883F8013D
:10128000F48089E794E06F2D0E94A92CEF2DF0E007
:10129000888190E0E827F927ED54FD4F808188830D
:1012A000F8012481358146815781232F342F452F22
:1012B0005527F22E89E794E0622F0E94A92CEF2D8A
:1012C000F0E0888190E0E827F927ED54FD4F808118
:1012D0008883F80124813581468157819A0144270A
:1012E0005527F22E89E794E0622F0E94A92CEF2D5A
:1012F000F0E0888190E0E827F927ED54FD4F8081E8
:101300008883F8012481358146815781252F332731
:1013100044275527F22E89E794E0622F0E94A92CDA
:10132000EF2DF0E0888190E0E827F927ED54FD4F9C
:101330008081888389E794E060E00E94A92CE8819D
:10134000F0E0ED54FD4F8081888389E794E060E010
:101350000E94A92CE881F0E0ED54FD4F8081888344
:10136000F801828193810B9718F18AE0A82EB12CA5
:10137000A00EB11E750112C0F701D1907F0189E75F
:1013800094E06D2D0E94A92CED2DF0E0888190E075
:10139000E827F927ED54FD4F808188832E2D2A19E7
:1013A00030E0F801828193810A972817390720F3EA
:1013B000075F1E4F89E794E0F80160810E94A92C25
:1013C000DF91CF911F910F91FF90EF90DF90BF9031
:1013D000AF900895DF93CF93CDB7DEB7CA50D14019
:1013E0000FB6F894DEBF0FBECDBF2CE329836A830E
:1013F0002AE030E03C832B83FC0184819581A68127
:10140000B7818D839E83AF83B887CE0101960E94FA
:10141000EE08C65FDE4F0FB6F894DEBF0FBECDBF3D
:10142000CF91DF9108958FE896E06AE773E00E941C
:101430005832882331F586E696E6A6E6B0E4809336
:10144000030690930406A0930506B093060680E079
:1014500090E0A0E8BFE38093070690930806A0936E
:101460000906B0930A0688EE93E090930C068093E9
:101470000B0681E880930D068DE880930E068DEFB4
:1014800025C082E598EBAEE0B0E48093030690932C
:101490000406A0930506B093060685E89BEEA1E539
:1014A000B0E48093070690930806A0930906B093D2
:1014B0000A0680EA94E190930C0680930B068BEF6A
:1014C00080930D0686E680930E068AEF80930F06C2
:1014D0000895FF920F931F930FE816E0C8016CE781
:1014E00073E00E94583280935C06C8016EE773E097
:1014F0000E94583280935D06C80160E873E00E9444
:10150000583280933606C8016EE873E00E94583264
:1015100080935406C8016AE873E00E9458328093B1
:101520005206C80164E873E00E94583280935E0658
:10153000C80166E873E00E94583280935F06C801D4
:101540006CE873E00E94583280934406C80162E957
:1015500073E00E94583280936006C80164E973E02A
:101560000E94583280934306C80164EF73E00E94E2
:101570005832F82EC80165EF73E00E945832382FB8
:1015800020E02F0D311D3093380620933706C80117
:1015900066EF73E00E945832F82EC80167EF73E0DF
:1015A0000E945832382F20E02F0D311D30933C0619
:1015B00020933B06C80168EF73E00E945832F82E72
:1015C000C80169EF73E00E945832382F20E02F0DD8
:1015D000311D30933A0620933906C8016BEF73E052
:1015E0000E945832809335061F910F91FF90089505
:1015F000BC018FE896E00E94583208956091C804BB
:101600007091C9048091CA049091CB0420E030E02D
:1016100040E152E40E94D33720E030E044EB53E451
:101620000E9405360E9436380E946D369B01255077
:10163000304037FF03C09B01215E3F4FAAE1B6E077
:10164000F901ED54FC4F80818C932F5F3F4F243282
:10165000310514F020E030E0119686E0A532B8079D
:1016600079F71C9208952F923F924F925F926F925A
:101670007F928F929F92AF92BF92CF92DF92EF9222
:10168000FF920F931F93DF93CF9300D000D000D031
:10169000CDB7DEB7182F662E2091BE043091BF045F
:1016A0002A35310530F0C9018D549F4F8935910598
:1016B000E8F437FF02C02D543F4FC90137FF03C084
:1016C000909581959F4F8A3191053CF0F4E48F2EDF
:1016D000912CE9ED2E2E312C1DC00A975CF17BE395
:1016E000872E912C62ED262E312C20C02B35310512
:1016F00014F0235B3040C90137FF03C090958195FA
:101700009F4F8A31910554F056E5852E912C4CED72
:10171000242E312C37E0A32EB12C15C00A9754F09B
:101720002DE4822E912C94ED292E312C88E0A82EC8
:10173000B12C09C005E0802E912CB8E32B2E312C62
:10174000A9E0AA2EB12C6091C0047091C104882731
:1017500077FD8095982F0E94A03627EA32E94BE268
:101760005CEB0E94D3370E94A73820E030E040EACB
:1017700050E40E94D33720E030E040E951E40E9479
:10178000D3370E94363820E030E044E352E40E9430
:1017900038350E946D36712EFEEBCF2EFFEFDF2E17
:1017A0009B01442737FD4095542F29833A834B836F
:1017B0005C83E6E94E2EE4E05E2E4AEF5FEF240EF6
:1017C000351E6091BE047091BF04882777FD809517
:1017D000982F0E94A03625E33AEF4EE85CE30E9482
:1017E000D3370E94A7387B018C01B601882777FD8B
:1017F0008095982F0E94A0369B01AC01C801B701CB
:101800000E94D3377B018C0169817A818B819C8115
:101810000E94A0369B01AC01C801B7010E94383577
:101820000E946D369B01CB0101978A35910508F026
:1018300071C062E170E00E94F9388B012F5F3F4F69
:10184000AEEEBFEF6A9FC0016B9F900D7A9F900D27
:101850001124820F931F62E070E00E94F9386D83BB
:101860007E83E62CE01A4E2D4C5F86E994E0672DCE
:101870000E942F0500D000D000D0EDB7FEB7319602
:10188000ADB7BEB712965C924E92119720E031E050
:10189000338322838D819E81880D991D9583848356
:1018A0000E94A72B4DB75EB74A5F5F4F0FB6F89403
:1018B0005EBF0FBE4DBF8D819E818A159B0554F181
:1018C000043011053CF593E0E90EC201672D4E2D61
:1018D0000E942F0500D000D000D0EDB7FEB73196A2
:1018E000ADB7BEB712965C924E92119720E031E0F0
:1018F000338322834D815E81420D531D5583448382
:101900000E94A72B8DB79EB706960FB6F8949EBF80
:101910000FBE8DBFACE0B0E0CA0EDB1E7394BEE418
:10192000CB16D10409F04DCF26960FB6F894DEBF42
:101930000FBECDBFCF91DF911F910F91FF90EF9020
:10194000DF90CF90BF90AF909F908F907F906F90DF
:101950005F904F903F902F900895823010F422E0D6
:1019600002C0282F220F30E08DB79EB708970FB620
:10197000F8949EBF0FBE8DBFEDB7FEB7319686E9D6
:1019800094E0ADB7BEB712969C938E93119783E007
:1019900091E09383828322573F4F358324832F5FC7
:1019A0003F4F378326830E94A72B8DB79EB708969B
:1019B0000FB6F8949EBF0FBE8DBF0895CF93DF93EF
:1019C000AC01E091D004F091D10420911006309147
:1019D0001106C9018C599F4F8E179F071CF4EA010D
:1019E000219709C024563040E217F30714F0EA01AA
:1019F00002C0EA012196842F90E0C817D90729F088
:101A00008FE896E04C2F0E945F32CE01DF91CF919C
:101A100008950F931F930FE816E0C80163EF73E07A
:101A200041E00E945F32C80164EF73E043E10E942D
:101A30005F32C80165EF73E046E00E945F32C80183
:101A400066EF73E040E10E945F32C80167EF73E028
:101A500047E20E945F32C80168EF73E048E80E94E5
:101A60005F32C80169EF73E043E10E945F321F916A
:101A70000F910895CF92DF92EF92FF920F931F93F1
:101A8000CF93DF937C016B01EA0100D000D006E91F
:101A900014E0EDB7FEB7128301838FED90E09483DD
:101AA00083830E94962B0F900F900F900F90CA3057
:101AB000D10581F0C436D10521F0C130D10519F529
:101AC00012C000D000D0EDB7FEB7128301838DEDB8
:101AD00090E011C000D000D0EDB7FEB712830183B3
:101AE0008AED90E008C000D000D0EDB7FEB71283B9
:101AF000018386ED90E0948383830E94962B0F9060
:101B00000F900F900F904091D0045091D1042091EC
:101B1000100630911106C9018C599F4F8417950703
:101B20002CF4C7018C1B9D0BEC0109C024563040DE
:101B30004217530714F0E70114C0CE0DDF1DCE1578
:101B4000DF0579F08FE896E0B6014C2F0E945F32F6
:101B50000894C11CD11C8FE896E0B6014D2F0E945D
:101B60005F32CE01DF91CF911F910F91FF90EF90E7
:101B7000DF90CF900895CF92DF92EF92FF920F9374
:101B80001F937C01D62EC72E06E914E0C8016E2DE6
:101B90004D2D0E949804C8010E94700500D000D00D
:101BA000EDB7FEB71283018383E391E094838383CF
:101BB0000E94962BEDB7FEB71283018383E291E07A
:101BC000948383830E94962BEDB7FEB71283018323
:101BD00083E191E0948383830E94962BEDB7FEB757
:101BE0001283018383E091E0948383830E94962B88
:101BF000EDB7FEB71283018384EF90E09483838373
:101C00000E94962B0F900F900F900F90C8010E948A
:101C10005405C70101966D2D7C2D0E94330B1F9139
:101C20000F91FF90EF90DF90CF900895AF92BF9209
:101C3000CF92DF92EF92FF920F931F93B82EA62EB2
:101C40000E94403328EE33E040E050E00E940C391F
:101C500069017A0106E914E0C8016B2D4A2D0E9442
:101C60009804C8010E9470058DB79EB70C970FB6F7
:101C7000F8949EBF0FBE8DBFEDB7FEB73196ADB7DE
:101C8000BEB712961C930E93119788E091E0938350
:101C9000828383EB90E095838483C6016CE370E0DC
:101CA0000E94F938CB016CE370E00E94F938978309
:101CB00086838AE390E091878087C6016CE370E0B9
:101CC0000E94F938938782870E94A72B8DB79EB711
:101CD0000C960FB6F8949EBF0FBE8DBFC8010E9430
:101CE00054051F910F91FF90EF90DF90CF90BF9020
:101CF000AF9008950F931F93282F462F06E914E005
:101D0000C801622F0E949804C8010E94700500D08B
:101D100000D0EDB7FEB71283018384E191E0948394
:101D200083830E94A72B0F900F900F900F90C801F4
:101D30000E9454051F910F9108958F929F92AF9228
:101D4000BF92CF92DF92EF92FF920F931F93E82EF4
:101D5000F62E06E914E0C8016E2D4F2D0E9498045E
:101D6000C8010E9470058DB79EB70C970FB6F89406
:101D70009EBF0FBE8DBFEDB7FEB73196ADB7BEB7F4
:101D800012961C930E9311978CE1882E81E0982E69
:101D900093828282BDEEAB2EB12CB582A48280915B
:101DA000E7049091E804A091E904B091EA048683E5
:101DB0009783A087B187A3EFCA2ED12CD386C28682
:101DC0000E94A72B8DB79EB70C960FB6F8949EBFB6
:101DD0000FBE8DBFC8010E945405F394C8016E2D3B
:101DE0004F2D0E949804C8010E947005ADB7BEB780
:101DF0001C970FB6F894BEBF0FBEADBFEDB7FEB7D0
:101E0000319612961C930E93119793828282B5821B
:101E1000A4828091EB049091EC04A091ED04B09128
:101E2000EE0486839783A087B187D386C2860E94FB
:101E3000A72B8DB79EB70C960FB6F8949EBF0FBE1A
:101E40008DBFC8010E945405F394C8016E2D4F2D1B
:101E50000E949804C8010E947005ADB7BEB71C97D8
:101E60000FB6F894BEBF0FBEADBFEDB7FEB731964B
:101E700012961C930E93119793828282B582A4824C
:101E80008091EF049091F004A091F104B091F204DC
:101E900086839783A087B187D386C2860E94A72BAB
:101EA0008DB79EB70C960FB6F8949EBF0FBE8DBF30
:101EB000C8010E9454051F910F91FF90EF90DF9091
:101EC000CF90BF90AF909F908F9008950F931F93E6
:101ED000282F462F06E914E0C801622F0E949804BB
:101EE000C8010E9470058DB79EB70A970FB6F89487
:101EF0009EBF0FBE8DBFEDB7FEB73196ADB7BEB773
:101F000012961C930E93119786E291E0938382833D
:101F100089EB90E09583848380911206909113065B
:101F20009783868382E890E0918780870E94A72B21
:101F30008DB79EB70A960FB6F8949EBF0FBE8DBFA1
:101F4000C8010E9454051F910F910895EF92FF92CE
:101F50000F931F93282F462F96E9E92E94E0F92E30
:101F6000C701622F0E949804C7010E9470058DB7B7
:101F70009EB70C970FB6F8949EBF0FBE8DBF0DB7DE
:101F80001EB70F5F1F4FEDB7FEB7F282E1828EE200
:101F900091E0F8019383828384EE90E095838483BB
:101FA0006091140670911506882777FD8095982F0B
:101FB0000E94A0362AE037ED43E25CE30E94D3376B
:101FC000F80166837783808791878FE890E0938715
:101FD00082870E94A72B8DB79EB70C960FB6F894F8
:101FE0009EBF0FBE8DBFC7010E9454051F910F9168
:101FF000FF90EF9008950F931F93282F462F06E927
:1020000014E0C801622F0E949804C8010E94700564
:102010008DB79EB70C970FB6F8949EBF0FBE8DBFBD
:10202000EDB7FEB73196ADB7BEB712961C930E93BF
:1020300011978EE291E09383828382EE90E0958304
:1020400084838091160690911706A0911806B0918E
:10205000190686839783A087B1878EE890E09387DF
:1020600082870E94A72B8DB79EB70C960FB6F89467
:102070009EBF0FBE8DBFC8010E9454051F910F91D6
:1020800008950F931F93282F462F86E994E0622F1F
:102090000E94980486E994E00E9470058091CD0426
:1020A000882319F428E331E057C0813019F42CE378
:1020B00031E052C0823019F420E431E04DC0833069
:1020C00019F424E431E048C0843019F428E431E004
:1020D00043C0853019F42CE431E03EC0863019F459
:1020E00020E531E039C0873019F424E531E034C00F
:1020F000883019F428E531E02FC0893019F42CE537
:1021000031E02AC08A3019F420E631E025C08B3056
:1021100019F424E631E020C08C3019F428E631E0CF
:102120001BC08D3019F42CE631E016C08E3019F446
:1021300020E731E011C08F3019F424E731E00CC002
:10214000803119F428E731E007C0813119F02CE71C
:1021500031E002C02DE731E08DB79EB708970FB68A
:10216000F8949EBF0FBE8DBFEDB7FEB7319606E95E
:1021700014E0ADB7BEB712961C930E93119781E889
:1021800091E09383828380EE90E09583848337830C
:1021900026830E94A72B8DB79EB708960FB6F8949A
:1021A0009EBF0FBE8DBFC8010E9454051F910F91A5
:1021B00008950F931F93282F462F06E914E0C801B6
:1021C000622F0E949804C8010E9470058DB79EB7C7
:1021D0000A970FB6F8949EBF0FBE8DBFEDB7FEB73E
:1021E0003196ADB7BEB712961C930E93119786E841
:1021F00091E09383828387E890E095838483809144
:10220000CE049091CF049783868385E290E09187F6
:1022100080870E94A72B8DB79EB70A960FB6F894B9
:102220009EBF0FBE8DBFC8010E9454051F910F9124
:1022300008950F931F93282F462F06E914E0C80135
:10224000622F0E949804C8010E9470058DB79EB746
:102250000A970FB6F8949EBF0FBE8DBFEDB7FEB7BD
:102260003196ADB7BEB712961C930E93119780E9C5
:1022700091E0938382838091C0049091C1049583FF
:10228000848380EB90E09783868381EB90E0918755
:1022900080870E94A72B8DB79EB70A960FB6F89439
:1022A0009EBF0FBE8DBFC8010E9454051F910F91A4
:1022B00008950F931F93282F462F06E914E0C801B5
:1022C000622F0E949804C8010E9470058DB79EB7C6
:1022D0000A970FB6F8949EBF0FBE8DBFEDB7FEB73D
:1022E0003196ADB7BEB712961C930E93119780E945
:1022F00091E0938382838091BE049091BF04958383
:10230000848380EB90E09783868382EB90E09187D3
:1023100080870E94A72B8DB79EB70A960FB6F894B8
:102320009EBF0FBE8DBFC8010E9454051F910F9123
:1023300008950F931F93282F462F06E914E0C80134
:10234000622F0E949804C8010E9470058DB79EB745
:102350000A970FB6F8949EBF0FBE8DBFEDB7FEB7BC
:102360003196ADB7BEB712961C930E93119788E9BC
:1023700091E09383828381EE90E0958384838091C2
:102380009802909199029783868385E290E09187E5
:1023900080870E94A72B8DB79EB70A960FB6F89438
:1023A0009EBF0FBE8DBFC8010E9454051F910F91A3
:1023B00008950F931F93282F462F06E914E0C801B4
:1023C000622F0E949804C8010E9470058DB79EB7C5
:1023D0000C970FB6F8949EBF0FBE8DBFEDB7FEB73A
:1023E0003196ADB7BEB712961C930E93119780EA43
:1023F00091E0938382838AEA91E09583848380EDE0
:1024000090E0978386838AE196E09187808781EDCB
:1024100090E0938782870E94A72B8DB79EB70C967A
:102420000FB6F8949EBF0FBE8DBFC8010E94540521
:102430001F910F9108950F931F93282F462F06E9A0
:1024400014E0C801622F0E949804C8010E94700520
:102450008DB79EB70A970FB6F8949EBF0FBE8DBF7B
:10246000EDB7FEB73196ADB7BEB712961C930E937B
:10247000119788EB91E0938382838091C8049091B7
:10248000C904A091CA04B091CB0484839583A68328
:10249000B78380EB90E0918780870E94A72B8DB750
:1024A0009EB70A960FB6F8949EBF0FBE8DBFC801A7
:1024B0000E9454051F910F9108950F931F93282F89
:1024C000462F06E914E0C801622F0E949804C80153
:1024D0000E9470058DB79EB70C970FB6F8949EBFFB
:1024E0000FBE8DBFEDB7FEB73196ADB7BEB7129632
:1024F0001C930E93119780EC91E09383828386E185
:1025000090E0958384838091E2049091E304A0910C
:10251000E404B091E50486839783A087B18788E8B7
:1025200090E0938782870E94A72B8DB79EB70C9669
:102530000FB6F8949EBF0FBE8DBFC8010E94540510
:102540001F910F910895EF92FF920F931F93282FE1
:10255000462F36E9E32E34E0F32EC701622F0E94A6
:102560009804C7010E9470058DB79EB70C970FB6EF
:10257000F8949EBF0FBE8DBF0DB71EB70F5F1F4FE4
:10258000EDB7FEB7F282E18280EC91E0F80193832F
:10259000828389EE90E0958384836091DE0470915C
:1025A000DF048091E0049091E104209103063091D2
:1025B000040640910506509106060E94D337F801A3
:1025C000668377838087918780910D068287138643
:1025D0000E94A72B8DB79EB70C960FB6F8949EBF9E
:1025E0000FBE8DBFC7010E9454051F910F91FF9030
:1025F000EF900895EF92FF920F931F93282F462F8D
:1026000056E9E52E54E0F52EC701622F0E9498048A
:10261000C7010E9470058DB79EB70C970FB6F8944E
:102620009EBF0FBE8DBF0DB71EB70F5F1F4FEDB71B
:10263000FEB7F282E1828AEC91E0F8019383828313
:1026400086EE90E0958384836091DA047091DB04D8
:102650008091DC049091DD042091070630910806FA
:102660004091090650910A060E94D337F80166830B
:1026700077838087918780910E06828713860E94D8
:10268000A72B8DB79EB70C960FB6F8949EBF0FBEC2
:102690008DBFC7010E9454051F910F91FF90EF90CD
:1026A0000895EF92FF920F931F93282F462F66E90C
:1026B000E62E64E0F62EC701622F0E949804C7013F
:1026C0000E9470058DB79EB70C970FB6F8949EBF09
:1026D0000FBE8DBF0DB71EB70F5F1F4FEDB7FEB713
:1026E000F282E1828AEC91E0F8019383828387EEA3
:1026F00090E0958384836091DA047091DB0480918B
:10270000DC049091DD0420912A0630912B06409143
:102710002C0650912D060E943735209107063091E6
:1027200008064091090650910A060E94D337F80125
:10273000668377838087918780910E0682871386D0
:102740000E94A72B8DB79EB70C960FB6F8949EBF2C
:102750000FBE8DBFC7010E9454051F910F91FF90BE
:10276000EF9008950F931F93282F462F06E914E04A
:10277000C801622F0E949804C8010E9470058091D0
:102780002E060E94AD0CC8010E9454051F910F91A6
:102790000895EF92FF920F931F93282F462F76E90B
:1027A000E72E74E0F72EC701622F0E949804C7013C
:1027B0000E9470058DB79EB70C970FB6F8949EBF18
:1027C0000FBE8DBF0DB71EB70F5F1F4FEDB7FEB722
:1027D000F282E1828AEC91E0F801938382838FE1B7
:1027E00090E09583848360912F06709130068091EC
:1027F0003106909132060E94A03620910706309152
:1028000008064091090650910A060E94D337F80144
:10281000668377838087918780910E0682871386EF
:102820000E94A72B8DB79EB70C960FB6F8949EBF4B
:102830000FBE8DBFC7010E9454051F910F91FF90DD
:10284000EF9008950F931F93282F462F06E914E069
:10285000C801622F0E949804C8010E9470058DB7BC
:102860009EB740970FB6F8949EBF0FBE8DBFEDB7D1
:10287000FEB73196ADB7BEB712961C930E93119763
:1028800084ED91E09383828383E890E09583848351
:102890008091C4049091C504A091C604B091C7046E
:1028A00086839783A087B18784E890E093878287A7
:1028B0008091D4049091D504A091D604B091D7040E
:1028C00084879587A687B7870E94A72B8DB79EB769
:1028D00040960FB6F8949EBF0FBE8DBFC8010E94F0
:1028E00054051F910F9108950F931F93282F462F82
:1028F00086E994E0622F0E94980486E994E00E94A1
:1029000070058091D904282F30E0823030F4E4E063
:10291000220F331FEA95E1F702C02150304000D06A
:1029200000D000D0EDB7FEB7319606E914E0ADB7A0
:10293000BEB712961C930E93119780E091E093839B
:102940008283358324830E94A72B8DB79EB706967A
:102950000FB6F8949EBF0FBE8DBFC8010E945405EC
:102960001F910F9108950F931F93282F462F06E96B
:1029700014E0C801622F0E949804C8010E947005EB
:102980008DB79EB708970FB6F8949EBF0FBE8DBF48
:10299000EDB7FEB73196ADB7BEB712961C930E9346
:1029A000119786EE91E0938382838FE090E0958388
:1029B00084838091D804868317820E94A72B8DB7C9
:1029C0009EB708960FB6F8949EBF0FBE8DBFC80184
:1029D0000E9454051F910F9108950F931F9306E9CC
:1029E00014E0C80163E045E00E949804C8010E9419
:1029F000700500D000D0EDB7FEB7128301838EE5DD
:102A000091E0948383830E94962BEDB7FEB71283E7
:102A100001838AE491E0948383830E94962BEDB72F
:102A2000FEB71283018383E491E0948383830E9441
:102A3000962B0F900F900F900F90C8010E94540595
:102A40001F910F9108950F931F93282F462F06E98A
:102A500014E0C801622F0E949804C8010E9470050A
:102A600000D000D0EDB7FEB71283018385E791E077
:102A7000948383830E94962B0F900F900F900F905A
:102A8000C8010E9454051F910F910895EF92FF9283
:102A90000F931F93CF93DF930E94403320913E0604
:102AA00030913F0640914006509141062617370766
:102AB0004807590708F04FC30E9440336C507E4FBF
:102AC0008F4F9F4F60933E0670933F068093400662
:102AD0009093410606E914E0C8010E94BD05C801B3
:102AE00065E043E00E949804C8010E94700500D090
:102AF00000D0ADB7BEB712961C930E93119786E225
:102B000092E014969C938E9313970E94962B0F90AD
:102B10000F900F900F908091100690911106892BC5
:102B200031F08091330690913406892B81F48091A5
:102B3000D0049091D1049093110680931006809157
:102B4000D2049091D304909334068093330620915D
:102B5000D2043091D3044091330650913406C90118
:102B6000845690404817590724F480913D068F5FA2
:102B700008C02C593F4F241735072CF480913D068F
:102B8000815080933D0680913D06181614F081E037
:102B900003C08D301CF08CE080933D0680913D0693
:102BA000863009F45AC187308CF4833009F4FAC0B6
:102BB000843034F4813079F1823009F0C8C28BC09E
:102BC0008430E9F0853009F0C2C222C0893009F4AE
:102BD000B7C18A3034F4873079F0883009F0B7C251
:102BE00014C08B3079F08B3024F08C3009F0AFC2F8
:102BF0002BC2C4E6D0E02FC2C4E6D0E0A8C1C4E630
:102C0000D0E032C184E690E021C284E690E09AC12F
:102C100084E690E024C100D000D0C6E9D4E0EDB74E
:102C2000FEB7D283C1838DE192E0948383830E94B7
:102C3000962B809101060F900F900F900F9080FFC0
:102C400026C000D000D0ADB7BEB71296DC93CE93AD
:102C5000119785E192E014969C938E9313970E94AE
:102C6000962B8091100690911106845690400F90FB
:102C70000F900F900F902091D0043091D10428171D
:102C800039070CF064C2809101068E7F21C000D00C
:102C900000D0EDB7FEB7D283C1838DE092E094837C
:102CA00083830E94962B80911006909111068C5977
:102CB0009F4F0F900F900F900F902091D004309164
:102CC000D104821793070CF042C280910106816003
:102CD000809301063CC200D000D0C6E9D4E0ADB775
:102CE000BEB71296DC93CE93119783E092E01496D0
:102CF0009C938E9313970E94962B0F900F900F909A
:102D00000F9080913506882301F100D000D0EDB7F7
:102D1000FEB7D283C18389EF91E0948383830E94BD
:102D2000962B8091100690911106845690400F903A
:102D30000F900F900F902091D0043091D10428175C
:102D400039073CF51092350624C000D000D0ADB74D
:102D5000BEB71296DC93CE9311978CEE91E0149649
:102D60009C938E9313970E94962B809110069091BE
:102D700011068C599F4F0F900F900F900F9020913C
:102D8000D0043091D104821793071CF481E0809322
:102D900035068FE896E06BEF73E0409135060E94B0
:102DA0005F32D5C100D000D0B6E9EB2EB4E0FB2EE7
:102DB000EDB7FEB7F282E1828BED91E094838383DD
:102DC0000E94962B8DB79EB708970FB6F8949EBFBA
:102DD0000FBE8DBF0DB71EB70F5F1F4FADB7BEB78C
:102DE0001296FC92EE9211978CEE91E0F80193838B
:102DF00082836091360670E080E090E00E949E360B
:102E000020E030E040E251E40E940536D8011496FB
:102E10006D937D938D939C93179786E790E0199619
:102E20009C938E93189780E290E01B969C938E93D0
:102E30001A970E94A72BEDB7FEB73C960FB6F894F1
:102E4000FEBF0FBEEDBF8091360690E060E873E0F4
:102E50000E94DE0C809336067AC18AE090E06AE038
:102E600070E00E94F938EB0100D000D006E914E0D0
:102E7000ADB7BEB712961C930E93119780EC91E0FC
:102E800014969C938E9313970E94962BEDB7FEB7E2
:102E900038970FB6F894FEBF0FBEEDBF3196ADB7B1
:102EA000BEB712961C930E9311978EE291E0938316
:102EB000828382EE90E095838483809116069091C0
:102EC0001706A0911806B091190686839783A087EC
:102ED000B1878EE890E0938782870E94A72BEDB799
:102EE000FEB736960FB6F894FEBF0FBEEDBF319613
:102EF000ADB7BEB712961C930E93119784EF91E075
:102F000093838283809137069091380695838483DA
:102F10000E94A72BEDB7FEB736960FB6F894FEBF0A
:102F20000FBEEDBF809137069091380664EF73E0D5
:102F3000AE010E943A0D909338068093370607C180
:102F40008AE090E06AE070E00E94F938EB0100D07E
:102F500000D0A6E9EA2EA4E0FA2EADB7BEB71296CD
:102F6000FC92EE92119785EA91E014969C938E93D1
:102F700013970E94962BEDB7FEB738970FB6F894CB
:102F8000FEBF0FBEEDBF0DB71EB70F5F1F4FF28222
:102F9000E1828EE291E0D80113969C938E93129772
:102FA00084EE90E015969C938E931497609114068E
:102FB00070911506882777FD8095982F0E94A0367E
:102FC0002AE037ED43E25CE30E94D337F8016683E1
:102FD0007783808791878FE890E0938782870E942C
:102FE000A72B8DB79EB706960FB6F8949EBF0FBE5F
:102FF0008DBFEDB7FEB73196ADB7BEB71296FC9256
:10300000EE9211978BE092E0938382838091390650
:1030100090913A06958384830E94A72BEDB7FEB763
:1030200036960FB6F894FEBF0FBEEDBF80913906FD
:1030300090913A0668EF73E0AE010E943A0D9093CA
:103040003A068093390683C08AE090E06AE070E037
:103050000E94F938EB0100D000D0F6E9EF2EF4E041
:10306000FF2EADB7BEB71296FC92EE9211978AE88A
:1030700091E014969C938E9313970E94962BEDB734
:10308000FEB738970FB6F894FEBF0FBEEDBF0DB771
:103090001EB70F5F1F4FF282E1828EE291E0D801EE
:1030A00013969C938E93129784EE90E015969C93C2
:1030B0008E9314976091140670911506882777FDFA
:1030C0008095982F0E94A0362AE037ED43E25CE31A
:1030D0000E94D337F80166837783808791878FE8D2
:1030E00090E0938782870E94A72B8DB79EB70696A4
:1030F0000FB6F8949EBF0FBE8DBFEDB7FEB73196E9
:10310000ADB7BEB71296FC92EE92119782E292E0B2
:103110009383828380913B0690913C0695838483C0
:103120000E94A72BEDB7FEB736960FB6F894FEBFF8
:103130000FBEEDBF80913B0690913C0666EF73E0B9
:10314000AE010E943A0D90933C0680933B0686E9BF
:1031500094E00E945405DF91CF911F910F91FF9051
:10316000EF9008952F923F924F925F926F927F92CD
:103170008F929F92AF92BF92CF92DF92EF92FF9287
:103180000F931F93DF93CF93CDB7DEB729970FB679
:10319000F894DEBF0FBECDBF8E836F830E94403395
:1031A00020914B0630914C0640914D0650914E06B1
:1031B000261737074807590708F02DC180914F0699
:1031C0008823C9F080939A0210924F0689E392E017
:1031D00090935106809350060E9440336C507E4F6E
:1031E0008F4F9F4F60934B0670934C0680934D0614
:1031F00090934E06CBC080919A02482E5524209180
:10320000CC042D8300915006109151068091B90491
:1032100089839091D9049C83A0914206AB838090CE
:10322000160690901706A0901806B0901906809187
:10323000360690E0609098027090990220914306C3
:10324000222E3324B0914406BA83598648866C01F5
:10325000EE24D7FCE094FE2CE885F9853196F987B9
:10326000E88736972CF081E090E09987888718C02E
:10327000A885B985A330B10509F1A430B1053CF4A6
:10328000A130B10569F0129709F047C010C0E88578
:10329000F985E430F105E1F0359709F03EC02EC024
:1032A000FD81F230D0F506E412E081E03DC02981D5
:1032B000233099F103E512E082E036C08C81823040
:1032C00060F59B81992349F100E612E083E02CC070
:1032D000C701B6010E94A03620E030E040E251E490
:1032E0000E9405369B01AC01C501B4010E94FE3568
:1032F00088239CF40DE612E084E016C06214730487
:1033000064F4ADE96A16AFEF7A0639F0BA81BB23EF
:1033100021F40AE712E085E007C0E885F985E415A5
:10332000F50509F099CF60C010935106009350063F
:1033300080934F0681E0809345060E944033685198
:103340007C4F8F4F9F4F60934B0670934C0680933A
:103350004D0690934E060E9440336056704F8F4F3B
:103360009F4F609347067093480680934906909359
:103370004A0680914606882321F086E994E00E945F
:10338000BD051092460602C01092450606E914E0FB
:10339000C8016E814F810E949804C8010E94700587
:1033A00000D000D000D0EDB7FEB73196ADB7BEB7B4
:1033B00012961C930E93119787E892E09383828371
:1033C0008091500690915106958384830E94A72B8B
:1033D000EDB7FEB736960FB6F894FEBF0FBEEDBF41
:1033E000C8010E94540517C010935106009350065F
:1033F00010924F060E9440332091470630914806B4
:103400004091490650914A06261737074807590741
:1034100008F4BACFBBCF29960FB6F894DEBF0FBE23
:10342000CDBFCF91DF911F910F91FF90EF90DF9073
:10343000CF90BF90AF909F908F907F906F905F9054
:103440004F903F902F900895EF92FF920F931F930C
:1034500080915206843009F056C09091CD0494308A
:1034600008F027C180915B068917A1F190935B0654
:103470000E94403360935706709358068093590614
:1034800090935A0690915B0680919B02981711F5D4
:1034900080914606813091F0813018F08230B1F48D
:1034A00013C011E0109346060E94403361537547E4
:1034B0008040904030F41093530608C082E080931F
:1034C00046061092530602C01092460686E994E022
:1034D0000E94BD050E944033209157063091580646
:1034E0004091590650915A06621B730B840B950B41
:1034F000615D77408040904008F4DBC08091CD044E
:1035000080939B02D6C0853029F4809190029091DF
:10351000910214C0863029F4809192029091930216
:103520000DC0873029F4809194029091950206C0D5
:10353000883041F4809196029091970290935606BC
:103540008093550680915406209155063091560679
:10355000882309F04AC0C901895097408F5A944086
:10356000C8F40E944033615375478040904020F476
:1035700081E0809353060CC080915306882341F468
:1035800080914506882321F486E994E00E94BD05D8
:1035900082E028C044E0203B340768F4809146066E
:1035A000882349F01092530686E994E00E94BD05F5
:1035B000109246067EC0205B34402955324008F008
:1035C00078C080914606813009F473C08091450629
:1035D000882309F06EC01092530686E994E00E9499
:1035E000BD0581E08093460664C0215B344008F449
:1035F00060C00E944033615375478040904008F09E
:1036000041C0809153068823E9F5E0905706F09079
:1036100058060091590610915A0688EE93E0A0E0F2
:10362000B0E0E80EF91E0A1F1B1F0E944033E61689
:10363000F70608071907E8F581E08093530617C0DD
:103640001092530686E994E00E94BD0580914606DB
:10365000823019F41092460603C08F5F80934606AD
:1036600080914606823018F082E0809346060E94E0
:103670004033609357067093580680935906909391
:103680005A0617C0E0905706F09058060091590668
:1036900010915A0688EE93E0A0E0B0E0E80EF91E23
:1036A0000A1F1B1F0E944033E616F706080719077A
:1036B00038F21F910F91FF90EF900895809152067C
:1036C000843010F00E94241A80915306882319F048
:1036D0000E94461508958091F90380FF08C060910B
:1036E0005F0480915D0490E070E00E94B2188091C8
:1036F0004606823008F0E8C1A82FB0E0FD01ED5089
:10370000FC4F808185FF0BC0FD01E15FFB4F6081B5
:10371000A35FBB4F8C9190E070E00E94B314809146
:103720004606A82FB0E0FD01ED50FC4F808186FFDA
:103730000BC0FD01ED5EFB4F6081AF5EBB4F8C9116
:1037400090E070E00E94741480914206882309F48E
:103750003FC080914606A82FB0E0FD01ED50FC4F20
:10376000808187FF0BC0FD01E95EFB4F6081AB5E8E
:10377000BB4F8C9190E070E00E942214809146062D
:10378000A82FB0E0FD01EB50FC4F808184FF0BC0FF
:10379000FD01E15DFB4F6081A35DBB4F8C9190E02B
:1037A00070E00E94C91380914606A82FB0E0FD0189
:1037B000EB50FC4F808183FF0BC0FD01E55DFB4FAB
:1037C0006081A75DBB4F8C9190E070E00E94B213C6
:1037D00080914206882309F483C08091D904823005
:1037E00008F47EC080914606A82FB0E0FD01E950A4
:1037F000FC4F808187FF0BC0FD01E95BFB4F6081BF
:10380000AB5BBB4F8C9190E070E00E9451138091B4
:103810004606A82FB0E0FD01E750FC4F808183FFF2
:103820000BC0FD01E959FB4F6081AB59BB4F8C9137
:1038300090E070E00E945D1280914606A82FB0E0F3
:10384000FD01E950FC4F808182FF0BC0FD01ED5B63
:10385000FB4F6081AF5BBB4F8C9190E070E00E94AA
:10386000FA1280914606A82FB0E0FD01E950FC4F06
:10387000808183FF0BC0FD01E55BFB4F6081A75B8F
:10388000BB4F8C9190E070E00E94A312809146069D
:10389000A82FB0E0FD01EB50FC4F808181FF0BC0F1
:1038A000FD01ED5DFB4F6081AF5DBB4F8C9190E002
:1038B00070E00E941B1280914606A82FB0E0FD0127
:1038C000EB50FC4F808180FF0BC0FD01E15EFB4FA0
:1038D0006081A35EBB4F8C9190E070E00E94D91193
:1038E00080914606A82FB0E0FD01E750FC4F808193
:1038F00086FF0BC0FD01E159FB4F6081A359BB4F0F
:103900008C9190E070E00E94991180914606A82F5A
:10391000B0E0FD01ED50FC4F808182FF0BC0FD0146
:10392000E95FFB4F6081AB5FBB4F8C9190E070E033
:103930000E94591180914606A82FB0E0FD01ED507C
:10394000FC4F808181FF0BC0FD01ED5FFB4F60816B
:10395000AF5FBB4F8C9190E070E00E941911809195
:103960004606A82FB0E0FD01E950FC4F808184FF9E
:103970000BC0FD01ED5AFB4F6081AF5ABB4F8C91DC
:1039800090E070E00E94D91080914606A82FB0E028
:10399000FD01E950FC4F808185FF0BC0FD01E95A14
:1039A000FB4F6081AB5ABB4F8C9190E070E00E945E
:1039B000411080914606A82FB0E0FD01ED50FC4F6C
:1039C000808183FF0BC0FD01E55FFB4F6081A75F36
:1039D000BB4F8C9190E070E00E94FB0F80914606F7
:1039E000A82FB0E0FD01E950FC4F808180FF0BC0A3
:1039F000FD01E15CFB4F6081A35CBB4F8C9190E0CB
:103A000070E00E94A60F80914606A82FB0E0FD014D
:103A1000ED50FC4F808184FF0BC0FD01E55EFB4F44
:103A20006081A75EBB4F8C9190E070E00E94660FB2
:103A300080914606A82FB0E0FD01E550FC4F808143
:103A400081FF18C080913506FD01EB58FB4F813096
:103A500049F4A958BB4F6C91808190E070E00E94BE
:103A60007A0E08C0A958BB4F6C91808190E070E03D
:103A70000E949D0E80914606A82FB0E0FD01EB50FC
:103A8000FC4F808187FF0BC0FD01E55CFB4F60812F
:103A9000A75CBB4F8C9190E070E00E94160E809165
:103AA0004606A82FB0E0FD01E950FC4F808186FF5B
:103AB0000BC0FD01E55AFB4F6081A75ABB4F8C91AB
:103AC00090E070E00E94BB0D089586E994E00E94AA
:103AD000BD050E94ED140E94130A0895CF93DF9351
:103AE000EC0186E994E00E949404C817D9073CF0E1
:103AF00086E994E00E948904892B09F42397CE017A
:103B0000DF91CF910895EF92FF920F931F93CF9380
:103B1000DF930091460610E08AEF90E0089F700165
:103B2000099FF00C189FF00C1124C7010E94F80A9D
:103B3000F801ED50FC4F882319F08081816002C0AC
:103B400080818E7F808380914606C82FD0E0C70198
:103B500002960E94F80AC350DC4F88838091460683
:103B6000C82FD0E0C70104960E94F80A90E00E9496
:103B70006E1DC150DC4F88830091460610E0C701DE
:103B800088569F4F0E94F80AF801ED50FC4F882399
:103B900019F08081806102C080818F7E8083809156
:103BA0004606C82FD0E0C70186569F4F0E94F80AEC
:103BB000C75EDB4F888380914606C82FD0E0C701DF
:103BC00084569F4F0E94F80A90E00E946E1DC55EC9
:103BD000DB4F88830091460610E0C70106960E94DD
:103BE000F80AF801ED50FC4F882319F080818260BB
:103BF00002C080818D7F808380914606C82FD0E0EF
:103C0000C70108960E94F80ACF5FDB4F8883809136
:103C10004606C82FD0E0C7010A960E94F80A90E035
:103C20000E946E1DCD5FDB4F88830091460610E039
:103C3000C7010C960E94F80AF801ED50FC4F88234A
:103C400019F08081846002C080818B7F80838091A5
:103C50004606C82FD0E0C7010E960E94F80ACB5F37
:103C6000DB4F888380914606C82FD0E0C70140967D
:103C70000E94F80A90E00E946E1DC95FDB4F8883A6
:103C80000091460610E0C70142960E94F80AF8012A
:103C9000ED50FC4F882319F08081886002C080813C
:103CA000877F808380914606C82FD0E0C701449665
:103CB0000E94F80AC75FDB4F888380914606C82FB1
:103CC000D0E0C70146960E94F80A90E00E946E1D5F
:103CD000C55FDB4F88830091460610E0C7014E9612
:103CE0000E94F80AF801ED50FC4F882319F08081FA
:103CF000806202C080818F7D808380914606C82FBC
:103D0000D0E0C70180960E94F80AC35FDB4F88832A
:103D100080914606C82FD0E0C70182960E94F80A1B
:103D200090E00E946E1DC15FDB4F888300914606C4
:103D300010E0C70184960E94F80AF801ED50FC4F8C
:103D4000882319F08081806402C080818F7B80830A
:103D500080914606C82FD0E0C70186960E94F80AD7
:103D6000CF5EDB4F888380914606C82FD0E0C70125
:103D700088960E94F80A90E00E946E1DCD5EDB4F8F
:103D800088830091460610E0C7018A960E94F80ACF
:103D9000F801ED50FC4F882319F08081806802C043
:103DA00080818F77808380914606C82FD0E0C7013D
:103DB0008C960E94F80ACB5EDB4F88838091460682
:103DC000C82FD0E0C7018E960E94F80A90E00E94AA
:103DD0006E1DC95EDB4F88830091460610E0C70167
:103DE000C0960E94F80AF801EB50FC4F882319F0A6
:103DF0008081816002C080818E7F808380914606B1
:103E0000C82FD0E0C701C2960E94F80AC35EDB4FFC
:103E1000888380914606C82FD0E0C701C4960E94CF
:103E2000F80A90E00E946E1DC15EDB4F888300910E
:103E3000460610E0C701C6960E94F80AF801EB504A
:103E4000FC4F882319F08081826002C080818D7FC1
:103E5000808380914606C82FD0E0C701C8960E9493
:103E6000F80ACF5DDB4F888380914606C82FD0E0EB
:103E7000C701CA960E94F80A90E00E946E1DCD5DAF
:103E8000DB4F88830091460610E0C701CC960E9464
:103E9000F80AF801EB50FC4F882319F08081846008
:103EA00002C080818B7F808380914606C82FD0E03E
:103EB000C701CE960E94F80ACB5DDB4F88838091C4
:103EC0004606C82FD0E0C701805C9F4F0E94F80AC9
:103ED00090E00E946E1DC95DDB4F8883009146060D
:103EE00010E0C701885B9F4F0E94F80AF801EB5071
:103EF000FC4F882319F08081806102C080818F7E11
:103F0000808380914606C82FD0E0C701865B9F4F13
:103F10000E94F80AC35DDB4F888380914606C82F54
:103F2000D0E0C701845B9F4F0E94F80A90E00E9496
:103F30006E1DC15DDB4F88830091460610E0C7010E
:103F40008E5B9F4F0E94F80AF801EB50FC4F8823CC
:103F500019F08081886002C08081877F8083809192
:103F60004606C82FD0E0C7018C5B9F4F0E94F80A1D
:103F7000C75DDB4F888380914606C82FD0E0C7011C
:103F80008A5B9F4F0E94F80A90E00E946E1DC55DFB
:103F9000DB4F88830091460610E0C701805B9F4F8E
:103FA0000E94F80AF801EB50FC4F882319F0808139
:103FB000806202C080818F7D808380914606C82FF9
:103FC000D0E0C7018E5A9F4F0E94F80ACF5CDB4FAA
:103FD000888380914606C82FD0E0C7018C5A9F4F36
:103FE0000E94F80A90E00E946E1DCD5CDB4F888332
:103FF0000091460610E0C7018A5A9F4F0E94F80AB6
:10400000F801EB50FC4F882319F08081806402C0D6
:1040100080818F7B808380914606C82FD0E0C701C6
:10402000885A9F4F0E94F80ACB5CDB4F88838091AF
:104030004606C82FD0E0C701865A9F4F0E94F80A53
:1040400090E00E946E1DC95CDB4F8883009146069C
:1040500010E0C70182569F4F0E94F80AF801EB500A
:10406000FC4F882319F08081806802C080818F779F
:10407000808380914606C82FD0E0C70180569F4FAD
:104080000E94F80AC75CDB4F888380914606C82FE0
:10409000D0E0C7018E559F4F0E94F80A90E00E9421
:1040A0006E1DC55CDB4F88830091460610E0C7019A
:1040B0008E599F4F0E94F80AF801E950FC4F88235F
:1040C00019F08081816002C080818E7F8083809121
:1040D0004606C82FD0E0C7018C599F4F0E94F80AAE
:1040E000C35CDB4F888380914606C82FD0E0C701B0
:1040F0008A599F4F0E94F80A90E00E946E1DC15C91
:10410000DB4F88830091460610E0C70182599F4F1C
:104110000E94F80AF801E950FC4F882319F08081C9
:10412000846002C080818B7F808380914606C82F87
:10413000D0E0C70180599F4F0E94F80ACF5BDB4F48
:10414000888380914606C82FD0E0C7018E589F4FC4
:104150000E94F80A90E00E946E1DCD5BDB4F8883C1
:104160000091460610E0C70184579F4F0E94F80A4D
:10417000F801E950FC4F882319F08081806802C063
:1041800080818F77808380914606C82FD0E0C70159
:1041900082579F4F0E94F80ACB5BDB4F8883809148
:1041A0004606C82FD0E0C70180579F4F0E94F80AEB
:1041B00090E00E946E1DC95BDB4F8883009146062C
:1041C00010E0C7018E569F4F0E94F80AF801E9508F
:1041D000FC4F882319F08081826002C080818D7F2E
:1041E000808380914606C82FD0E0C7018C569F4F30
:1041F0000E94F80AC35BDB4F888380914606C82F74
:10420000D0E0C7018A569F4F0E94F80A90E00E94B2
:104210006E1DC15BDB4F88830091460610E0C7012D
:104220008C589F4F0E94F80AF801E950FC4F8823F0
:1042300019F08081886002C08081877F80838091AF
:104240004606C82FD0E0C7018A589F4F0E94F80A3F
:10425000C75BDB4F888380914606C82FD0E0C7013B
:1042600088589F4F0E94F80A90E00E946E1DC55B1F
:10427000DB4F88830091460610E0C70186589F4FA8
:104280000E94F80AF801E950FC4F882319F0808158
:10429000806102C080818F7E808380914606C82F16
:1042A000D0E0C70184589F4F0E94F80ACF5ADB4FD5
:1042B000888380914606C82FD0E0C70182589F4F5F
:1042C0000E94F80A90E00E946E1DCD5ADB4F888351
:1042D0000091460610E0C70180589F4F0E94F80ADF
:1042E000F801E950FC4F882319F08081806202C0F8
:1042F00080818F7D808380914606C82FD0E0C701E2
:104300008E579F4F0E94F80ACB5ADB4F88838091CB
:104310004606C82FD0E0C7018C579F4F0E94F80A6D
:1043200090E00E946E1DC95ADB4F888300914606BB
:1043300010E0C7018A579F4F0E94F80AF801E95020
:10434000FC4F882319F08081806402C080818F7BBC
:10435000808380914606C82FD0E0C70188579F4FC1
:104360000E94F80AC75ADB4F888380914606C82FFF
:10437000D0E0C70186579F4F0E94F80A90E00E9444
:104380006E1DC55ADB4F88830091460610E0C701B9
:104390008C559F4F0E94F80AF801E750FC4F882384
:1043A00019F08081816002C080818E7F808380913E
:1043B0004606C82FD0E0C7018A559F4F0E94F80AD1
:1043C000C35ADB4F888380914606C82FD0E0C701CF
:1043D00088559F4F0E94F80A90E00E946E1DC15AB6
:1043E000DB4F88830091460610E0C70180559F4F40
:1043F0000E94F80AF801E750FC4F882319F08081E9
:10440000846002C080818B7F808380914606C82FA4
:10441000D0E0C7018E549F4F0E94F80ACF59DB4F5E
:10442000888380914606C82FD0E0C7018C549F4FE7
:104430000E94F80A90E00E946E1DCD59DB4F8883E0
:104440000091460610E0C7018A549F4F0E94F80A67
:10445000F801E750FC4F882319F08081886002C082
:104460008081877F808380914606C82FD0E0C70176
:1044700088549F4F0E94F80ACB59DB4F8883809164
:104480004606C82FD0E0C70186549F4F0E94F80A05
:1044900090E00E946E1DC959DB4F8883009146064B
:1044A00010E0C70184549F4F0E94F80AF801E750BA
:1044B000FC4F882319F08081806102C080818F7E4B
:1044C000808380914606C82FD0E0C70182549F4F59
:1044D0000E94F80AC759DB4F888380914606C82F8F
:1044E000D0E0C70180549F4F0E94F80A90E00E94DC
:1044F0006E1DC559DB4F88830091460610E0C70149
:10450000845A9F4F0E94F80AF801E750FC4F882315
:1045100019F08081806402C080818F7B80838091CC
:104520004606C82FD0E0C701825A9F4F0E94F80A62
:10453000C359DB4F888380914606C82FD0E0C7015E
:10454000805A9F4F0E94F80A90E00E946E1DC15948
:10455000DB4F88830091460610E0C70180529F4FD1
:104560000E94F80AF801E550FC4F882319F0808179
:10457000846002C080818B7F808380914606C82F33
:10458000D0E0C7018E519F4F0E94F80ACF58DB4FF1
:10459000888380914606C82FD0E0C7018C519F4F79
:1045A0000E94F80A90E00E946E1DCD58DB4F888370
:1045B0000091460610E0C7018C529F4F0E94F80AF6
:1045C000F801E550FC4F882319F08081826002C019
:1045D00080818D7F808380914606C82FD0E0C701FF
:1045E0008A529F4F0E94F80ACB58DB4F88838091F4
:1045F0004606C82FD0E0C70188529F4F0E94F80A94
:1046000090E00E946E1DC958DB4F8883DF91CF91E7
:104610001F910F91FF90EF9008954F925F927F92BC
:104620008F929F92AF92BF92CF92DF92EF92FF92C2
:104630000F931F93DF93CF93CDB7DEB7C854D0400D
:104640000FB6F894DEBF0FBECDBF06E914E0C80177
:104650000E94BD05C80166E049E00E949804C801B7
:104660000E94700500D000D0EDB7FEB71283018321
:1046700081E592E0948383830E94962B0F900F90A4
:104680000F900F90C8010E94540500D000D009E798
:1046900014E0EDB7FEB71283018381E492E09483C6
:1046A00083830E94962B46E3442E42E0542EEE2450
:1046B000FF24CC24DD240F900F900F900F90702ECC
:1046C000012F39E0A32EB12CAC0EBD1E4E01089473
:1046D000811C911C89E794E00E944A2C982F8D3010
:1046E00031F08D30DCF180538230C0F530C01830AD
:1046F000A1F59981892F8053823078F5913311F497
:1047000090E801C090E08A81813309F4905C8B814C
:10471000813309F4905E8C81813309F4905F8D813F
:10472000813309F4985F8E81813309F49C5F8F8116
:10473000813309F49E5F8885813309F49F5FF50119
:10474000EE0DFF1D90830894E11CF11C06C0F401DE
:10475000E10FF11D90831F5F01C010E0F0E4EF1640
:10476000F104C9F486E994E0B601A5010E94A80409
:104770000894C11CD11C00D000D0EDB7FEB77182E7
:104780000283548243820E94962BEE24FF240F90D2
:104790000F900F900F90FFEFCF16D10409F00CF49B
:1047A00099CFC85BDF4F0FB6F894DEBF0FBECDBF09
:1047B000CF91DF911F910F91FF90EF90DF90CF90FD
:1047C000BF90AF909F908F907F905F904F90089593
:1047D000BF92CF92DF92EF92FF920F931F93DF93DE
:1047E000CF93CDB7DEB72E970FB6F894DEBF0FBECE
:1047F000CDBF73E0C72ED12CCC0EDD1E67E0E62EB8
:10480000F12CEC0EFD1E53E0B52E12C30E94403376
:1048100060527E4480409040C8F40E944033695802
:1048200073418040904090F01A3011F01D3031F407
:104830008091FD058F5F8093FD0502C01092FD05FC
:104840008091FD05833011F40E940D23812F63EFC9
:1048500074E00E941A07882311F400E0E3C28091FB
:10486000F7049091F804A091F904B091FA04863EFF
:1048700046EA940746E2A4074DE7B40709F4D3C11A
:10488000873E56EA950756E2A5075DE7B50708F0AB
:104890007CC08035EFED9E07EDEEAE07E8E1BE0788
:1048A00009F46DC28135FFED9F07FDEEAF07F8E11A
:1048B000BF0788F584302AE9920727EDA2072EE08A
:1048C000B20709F450C185303AE9930737EDA307E1
:1048D0003EE0B30780F486314AEA940747E3A40731
:1048E0004BE0B40709F43FC184559447A54CBB4045
:1048F00009F08EC224C28239E3EA9E07ECEEAE07CD
:10490000E4E1BE0709F42FC188599C42AA41B6418F
:1049100009F07EC231C1823D22EC920722E8A20753
:104920002EE1B20709F428C1833D32EC930732E847
:10493000A3073EE1B30780F48E3C48E4940747E5C3
:10494000A4074AE1B40709F46EC184579B4EAA47F5
:10495000BB4109F05DC207C1863EE5ED9E07EAED69
:10496000AE07E3E3BE0709F48BC08036FBED9F077B
:10497000FBE3AF07FEE6BF0709F4F5C088529E458A
:10498000A24DB44209F044C2EEC08A3837EF930713
:1049900037ECA30738EBB30709F4EEC08B3847EFC9
:1049A000940747ECA40748EBB40788F58C3855E822
:1049B000950757EAA50758E9B50709F434C18D38BA
:1049C000E5E89E07E7EAAE07E8E9BE0780F480382D
:1049D000FCED9F07F5E4AF07F2E8BF0709F4AFC1AC
:1049E00082559A4EA048BA4809F012C2BCC08E3710
:1049F00032E193073AE6A3073BE9B30709F4B3C0F2
:104A00008A57964FA14FBD4909F002C20CC18436A6
:104A100059ED950750EEA50757EDB50789F1853695
:104A2000E9ED9E07E0EEAE07E7EDBE0780F48038C3
:104A3000F4E79F07F0E1AF07F4ECBF0709F49CC06F
:104A400084559D42AF4FB54C09F0E2C18CC08E3405
:104A50003DE593073EE3A30733EEB30709F483C0B4
:104A6000823F4DEE940744E2A4074DEFB40709F4EA
:104A700081C1865B9342A34AB24E09F0C9C1D3C03B
:104A80000E9440336093BA047093BB048093BC04CB
:104A90009093BD04B092B90480910D0590910E05DC
:104AA000A0910F05B0911005F70180839183A28337
:104AB000B3836F81788589859A850E946D3670935E
:104AC000BF046093BE048091110590911205A091DE
:104AD0001305B0911405F70180839183A283B383FA
:104AE0006F81788589859A850E946D367093C1049F
:104AF0006093C0048091150590911605A09117054B
:104B0000B0911805F70180839183A283B3836F81ED
:104B1000788589859A850E946D368B017093C304D0
:104B20006093C2046091C4047091C5048091C6046E
:104B30009091C70420E030E040E050E00E94FE3554
:104B4000882379F4B801882777FD8095982F0E94F3
:104B5000A0366093C8047093C9048093CA049093EC
:104B6000CB0401E056C18091FD048093CC04809178
:104B7000FE048093CD044CC18091FD049091FE040D
:104B8000A091FF04B0910005F70180839183A28377
:104B9000B3836F81788589859A8520E030E048EC81
:104BA00052E40E94D3370E946D367093CF04609315
:104BB000CE04693C710520F01092CF041092CE040F
:104BC00080911705909118059093D1048093D0049B
:104BD0008091190590911A059093D3048093D20483
:104BE00080911D0590911E059093910280939002F3
:104BF00080912105909122059093930280939202D7
:104C000080912305909124059093950280939402BE
:104C100080912505909126059A8389839093970228
:104C200080939602F5C06091FD047091FE0480911E
:104C3000FF04909100050E94A03620E836E948E183
:104C40005BE40E9405366093C4047093C5048093AE
:104C5000C6049093C704609101057091020580918C
:104C6000030590910405D6016C9311967C931197DE
:104C700012968C93129713969C930E94A03620E86C
:104C800036E948E15BE40E9405366093D4047093F2
:104C9000D5048093D6049093D70480912205809305
:104CA000D804809121058093D90480910D059091BD
:104CB0000E05A0910F05B0911005F7018083918337
:104CC000A283B3838F819885A985BA858093C80410
:104CD0009093C904A093CA04B093CB0480910505B6
:104CE00090910605A0910705B091080580839183F6
:104CF000A283B3838F819885A985BA858093DA04CE
:104D00009093DB04A093DC04B093DD048091110543
:104D100090911205A0911305B091140580839183A1
:104D2000A283B3838F819885A985BA858093DE0499
:104D30009093DF04A093E004B093E10469C08091F4
:104D4000050590910605A0910705B0910805F701AA
:104D500080839183A283B3838F819885A985BA8547
:104D6000B0588093E2049093E304A093E404B093DA
:104D7000E5044EC08091FD048093E60449C0809113
:104D8000FD049091FE04A091FF04B0910005F7018D
:104D900080839183A283B3838F819885A985BA8507
:104DA0008093E7049093E804A093E904B093EA04A5
:104DB0008091010590910205A0910305B091040531
:104DC00080839183A283B3838F819885A985BA85D7
:104DD0008093EB049093EC04A093ED04B093EE0465
:104DE0008091050590910605A0910705B0910805F1
:104DF00080839183A283B3838F819885A985BA85A7
:104E00008093EF049093F004A093F104B093F20424
:104E100000E08091F404823229F483EF94E063E2AD
:104E20000E94EA098EEB90E00E94A733002341F52F
:104E300089E794E00E941A2C1816190604F589E7F0
:104E400094E00E944A2C182F8091B904882309F01D
:104E5000FDCCDCCC1092B90401E0802F90E02E96BE
:104E60000FB6F894DEBF0FBECDBFCF91DF911F917B
:104E70000F91FF90EF90DF90CF90BF90089500E0EA
:104E80002091BA043091BB044091BC045091BD0400
:104E9000205F384D4F4F5F4F2B873C874D875E8794
:104EA0000E9440332B853C854D855E85261737074C
:104EB0004807590778F2D1CF6F927F928F929F92D5
:104EC000AF92BF92CF92DF92EF92FF920F931F9318
:104ED000E0906106F090620600916306109164060E
:104EE0008FE590E0A0E0B0E0E80EF91E0A1F1B1F5E
:104EF0000E9440336E157F058007910708F427C193
:104F00000E9440333B014C01A0906106B0906206C4
:104F1000C0906306D09064060E944033609361069F
:104F200070936206809363069093640680E00E940B
:104F3000DC34AA2797FDA095BA2FBC01CD010E94B1
:104F4000A0362DEC3CEC4CE85FE30E94D33720E028
:104F500030E040E85AE30E94D3377B018C01609136
:104F6000370670913806882777FD8095982F0E9424
:104F7000A03620E030E048EC52E40E9405369B0168
:104F8000AC01C801B7010E94D3372DEC3CEC4CE4D6
:104F90005EE30E94D3377B018C0160919C0270918B
:104FA0009D0280919E0290919F022DEC3CEC4CE47E
:104FB0005FE30E94D3379B01AC01C801B7010E9497
:104FC0003835DC019B01AC0120939C0230939D029B
:104FD00040939E0250939F02CB01809316069093BC
:104FE0001706A0931806B093190680913B0690917E
:104FF0003C06181619060CF0AAC081E00E94DC34A9
:10500000AA2797FDA095BA2FBC01CD010E94A0361A
:105010002DEC3CEC4CE85FE30E94D33720E030E01D
:1050200040E85AE30E94D3377B018C016091390636
:1050300070913A06882777FD8095982F0E94A036B8
:1050400020E030E44CE156EC0E9405369B01AC01B7
:10505000C801B7010E9438357B018C0160913B0685
:1050600070913C06882777FD8095982F0E94A03686
:1050700020E030E048EC52E40E9405369B01AC0190
:10508000C801B7010E94D3372DEC3CEC4CE45EE341
:105090000E94D3377B018C016091690670916A068A
:1050A00080916B0690916C062DEC3CEC4CE45FE338
:1050B0000E94D3379B01AC01C801B7010E9438356B
:1050C0007B018C016093690670936A0680936B067E
:1050D00090936C06B3016A197B0980E090E00E940E
:1050E0009E369B01AC01C801B7010E94D3372FEA5D
:1050F00035EA41E959E30E94D337209165063091A2
:10510000660640916706509168060E9438355B013B
:105110006C016093650670936606809367069093B2
:105120006806C801B70120E030E048EC52E40E9474
:10513000D3370E946D367093150660931406C6012E
:10514000B5010E94723670931306609312061F9188
:105150000F91FF90EF90DF90CF90BF90AF909F9016
:105160008F907F906F900895EF92FF920F931F930F
:1051700080914406882351F083E00E94DC3464E08F
:1051800070E00E94F938609302063CC083E00E9400
:10519000DC34AA2797FDA095BA2FBC01CD010E944F
:1051A000A0362DEC3CEC4CE45EE30E94D33720E0CB
:1051B00030E040E85EE30E94D3377B018C016091D0
:1051C000020670E0882777FD8095982F0E94A03610
:1051D0002DEC3CEC4CE45FE30E94D3379B01AC0127
:1051E000C801B7010E9438350E94723620915F06CF
:1051F000621730F030915E06262F361708F4232F01
:10520000209302061F910F91FF90EF90089583E085
:105210000E94D934089583E00E94D93408951F93E1
:10522000CF93DF9385E090E06CE070E00E9423155F
:1052300068EE73E080E090E00E944E3389E794E0EE
:105240000E94972CC0E0D0E010E0CE016DE171E04B
:105250000E94F938892BA9F41F5E86E994E0612F3A
:105260004CE00E94980486E994E00E94700586E96B
:1052700094E06EEE0E94A00586E994E00E94540539
:10528000105161E070E080E090E00E944E33219682
:1052900087E0C13DD807C9F6DF91CF911F910895EE
:1052A00086E061E00E94853408950F931F9386E0A5
:1052B00061E00E94463409E714E0C80140E051EE85
:1052C00060E070E00E94B82B109391060093900666
:1052D0000E94502986E994E00E94F6050E94651D0F
:1052E00064EF71E080E090E00E944E3383EF93E042
:1052F0000E94F80A813011F00E94090D0E94690A8B
:105300001092460607C00E94831D809146068F5F5B
:1053100080934606809146068230A8F31092460696
:105320000E940F290E9407290E940B2988EA94E015
:1053300068E27BE224E630E040E050E000E00E94DA
:105340006B3286E994E00E94BD0588EA94E00E94F1
:10535000D1321F910F9108952F923F924F925F92F9
:105360006F927F928F929F92AF92BF92CF92DF9275
:10537000EF92FF920F931F93DF93CF9300D000D053
:10538000CDB7DEB780914206882309F4E1C0E090F2
:105390006D06F0906E0600916F0610917006C801C0
:1053A000B7019F7725E33AEF4EE85CE30E94D337DD
:1053B0000E94023669837A838B839C83C801B7017C
:1053C0002091C4043091C5044091C6045091C70493
:1053D0000E9437351B012C019F7720EC3BE649EDFD
:1053E00057E40E94D3375B016C01609171067091A4
:1053F000720680917306909174062091D4043091C6
:10540000D5044091D6045091D7040E9437353B0112
:105410004C019F7720EC3BE649ED57E40E94D337DF
:1054200029813A814B815C810E94D3377B018C01B9
:10543000C601B501A60195010E94D3375B016C013D
:10544000C801B701A80197010E94D3379B01AC01A5
:10545000C601B5010E9438350E945A380E946D3647
:1054600060932F0670933006809331069093320636
:1054700060E070E080E89FE329813A814B815C81A4
:105480000E9405369B01AC01C201B1010E94D337D5
:1054900097FA909497F89094A40193010E94AB35E9
:1054A00020EE3EE245E652E40E94D33720E030E0B1
:1054B00044EB52E40E9438350E946D369B01AC01EA
:1054C00097FF04C028593E4F4F4F5F4FCA01B901A3
:1054D000645B70408040904097FF06C0CA01B901EC
:1054E0006C547F4F8F4F9F4F0E94A0362091C8046D
:1054F0003091C9044091CA045091CB040E943735C1
:105500000E946D3697FF04C068597E4F8F4F9F4FA2
:105510000E94A03620E030E044EB53E40E940536C0
:1055200020E030E040E851E40E94D3370E94363852
:1055300020E030E040E85FE30E9438350E94723698
:1055400060932E06613108F46CC010922E0669C07B
:105550008091D904823008F464C08091D8048530E9
:1055600008F45FC0A09075068DE18A1508F459C053
:10557000E090DA04F090DB040091DC041091DD048B
:105580006091760670917706809178069091790601
:10559000A80197010E9437359F7720E030E040E076
:1055A0005FE30E94C83718165CF410927506E0920B
:1055B0007606F0927706009378061093790631C04C
:1055C0008A2D8F5F809375068E3159F58091C404C2
:1055D0009091C504A091C604B091C70480936D0654
:1055E00090936E06A0936F06B09370068091D404DA
:1055F0009091D504A091D604B091D7048093710600
:1056000090937206A0937306B0937406E0922A06F4
:10561000F0922B0600932C0610932D0681E08093C8
:1056200042060F900F900F900F90CF91DF911F9136
:105630000F91FF90EF90DF90CF90BF90AF909F9031
:105640008F907F906F905F904F903F902F90089534
:10565000CF92DF92EF92FF920F931F930E945C27ED
:105660000E94B42880910206282F30E030939902DE
:105670002093980280914406882359F500915F0693
:1056800010E0201B310BB901882777FD8095982FFA
:105690000E94A0366B017C0160915E0670E0601B89
:1056A000710B882777FD8095982F0E94A0369B016B
:1056B000AC01C701B6010E94053620E030E048EC9D
:1056C00052E40E94D3370E946D3670939902609322
:1056D000980280919802909199028D599F4F34F4CD
:1056E0008DE99FEF90939902809398020E9477082A
:1056F0000E94FE0A86E994E00E94AC290E945E1B8B
:105700001F910F91FF90EF90DF90CF9008950E942E
:10571000E823892B19F00E94282B089588EA94E049
:105720000E94B93208958FEF9FE70895DF93CF93DA
:10573000CDB7DEB7FE0139968D819E8161E04F8144
:1057400058859F010E94372ECF91DF910895DF93F6
:10575000CF93CDB7DEB7FE0139968D819E8160E093
:105760004F8158859F010E94372ECF91DF91089578
:105770000F931F93DC01ED91FC910288F389E02DDA
:1057800020E030E000E010E009951F910F910895AE
:105790008F92AF92CF92EF92FF920F931F93DF936E
:1057A000CF93CDB7DEB7FC011382128288EE93E06F
:1057B000A0E0B0E084839583A683B7838BED93E06C
:1057C000918380835587448737872687118B008B89
:1057D000F38AE28AC48AA58A868A70E0CB0123E034
:1057E000880F991F2A95E1F79C012258394F308F75
:1057F000278B8A57994F928F818F81E090E002C06A
:10580000880F991F6A95E2F720918E06282B209326
:105810008E06CF0140E051EE60E070E00E94B82BB0
:10582000CF91DF911F910F91FF90EF90CF90AF90AC
:105830008F900895FC01838D882319F42FEF3FEF9B
:105840000DC00788F08DE02D208131818281938108
:10585000281B390B8481958128233923C901089598
:10586000FC01838D882319F42FEF3FEF11C0018CC9
:10587000F28DE02D2081318182819381281B390BAB
:105880002095309584819581282339232F5F3F4FC0
:10589000C9010895FC01838D882361F0A789B08D2B
:1058A0002D913C91119712968D919C9113972817E9
:1058B000390721F44FEF5FEFCA01089512968D91D9
:1058C0009C9113971696ED91FC911797E80FF91F8D
:1058D000408112968D919C911397019614962D916B
:1058E0003C9115978223932313969C938E93129742
:1058F00050E0E2CFFC01838D882351F00788F08DC2
:10590000E02D20813181828193812817390721F48C
:105910002FEF3FEFC9010895828193810680F781BF
:10592000E02DE80FF91F8081282F30E0F3CFDC0154
:105930005796ED91FC915897828193819183808352
:105940005996ED91FC915A9780819181938382833E
:105950000895DC015B968C915B978823A9F1599699
:10596000ED91FC915A97208131812F5F3F4F8481C7
:105970009581282339235C968C915C97882329F0A4
:105980008281938128173907F9F082819381281742
:105990003907D9F3808191810680F781E02DE80FE6
:1059A000F91F60835996ED91FC915A9731832083BA
:1059B0005296ED91FC915397808156969C91892B3C
:1059C000808321E030E002C020E030E0C90108958A
:1059D000CF93DF93EC011B821A828A819B8199838A
:1059E00088831D821C828E819F81009721F00E94F6
:1059F000EA031F821E82DF91CF9108950F931F93B8
:105A00008C01DC015296ED91FC91539720815696C2
:105A10008C91569755969C915597892B809582230A
:105A2000808357968D919C9158970E94E82CF8019D
:105A3000818D928D0E94E82CD8015B961C921F915B
:105A40000F9108950F931F93CF93DF938C01FC0167
:105A500013821282828193819183808341E0A1E04D
:105A6000B0E001C04F5FFD01042E02C0EE0FFF1F2A
:105A70000A94E2F79B0182E06130780710F020E0A1
:105A800032E0E217F30770F3C1E0D0E002C0CC0FC0
:105A9000DD1F4A95E2F72197F8012681378121150C
:105AA000310541F0848195818C179D0789F0C901EA
:105AB0000E94EA03F801D583C483CE0101960E94B7
:105AC00040039C01F8019783868380E0232B09F033
:105AD00081E0DF91CF911F910F910895AF92BF9216
:105AE000CF92DF92EF92FF920F931F93CF93DF93AA
:105AF0007C015A016B01E901DC015B968C915B979B
:105B00008823F1F02115310539F45796ED91FC9178
:105B10005897C481D58121960115110549F4D70103
:105B20005996ED91FC915A97048115810F5F1F4F93
:105B3000D701ED91FC910088F189E02DC70109950D
:105B4000F7018789908D209711F4C0E8D0E0BE015D
:105B50000E94222D882381F0D70159968D919C9126
:105B60005A970115110511F400E110E0B8010E94E7
:105B7000222D882309F04DC0D701ED91FC910088BA
:105B8000F189E02DC701099567C0D7015096ED91C5
:105B9000FC915197B0E0AB16B1EEBB06B0E0CB067E
:105BA000B0E0DB0609F454C081E090E0D7015496E0
:105BB0000C9002C0880F991F0A94E2F7808360E07E
:105BC00079E08DE390E0A60195010E942E392150E5
:105BD000304040405040CA01B90122E030E040E08E
:105BE00050E00E942E39D7011C96ED91FC911D9733
:105BF00030831E96ED91FC911F972083D70152961A
:105C0000ED91FC915397808155969C91892B8083CF
:105C100023C0D7015996ED91FC915A9713821282B5
:105C200082819381918380835796ED91FC9158975F
:105C300013821282828193819183808381E05B96BB
:105C40008C931A141B041C041D040CF49ECFD6CF95
:105C5000108220E130E0C7CFDF91CF911F910F91EB
:105C6000FF90EF90DF90CF90BF90AF9008952F926C
:105C70003F924F925F926F927F928F929F92AF92DC
:105C8000BF92CF92DF92EF92FF920F931F93DF9319
:105C9000CF93CDB7DEB764970FB6F894DEBF0FBED3
:105CA000CDBF3C01688B5A8B498B69011C01AE0149
:105CB0004F5F5F4F5C8B4B8BE989FA89488940FDC8
:105CC000659140FF6191FA8BE98B662309F4D7C394
:105CD000653249F440FD859140FF8191FA8BE98B53
:105CE0008532B1F40CC06A3051F4D301ED91FC91CE
:105CF0000190F081E02DC1016DE009956AE0D301CA
:105D0000ED91FC910190F081E02DC1010995D4CF76
:105D1000982F10E0882499241032B0F49B3269F057
:105D20009C3228F4903251F0933271F40BC09D32C2
:105D300039F0903349F4116028C01260146025C016
:105D4000186023C0106121C017FD2BC0892F80531C
:105D50008A3078F416FF06C0BAE09B9E902C11247E
:105D6000980E13C0EAE08E9E802C1124880E1062DB
:105D70000CC09E3221F416FD82C3106406C09C360E
:105D800011F4106802C0983661F4E989FA894889EB
:105D900040FD959140FF9191FA8BE98B992309F091
:105DA000BBCF892F8554833020F4812F8061905E92
:105DB00007C0892F8556833008F0E6C1812F8F7E7A
:105DC00086FD02C076E0972E6FE3F62EF822953618
:105DD00019F450E4F52A07C0963619F480E8F82A39
:105DE00002C091109A94F7FE0BC09BE3991520F422
:105DF00027E05CE3B52E0DC0B92CB39427E009C0B1
:105E0000A7E0A91520F447E0942E27E001C0292D32
:105E1000BB24F6013496FD87EC87D6016D917D9108
:105E20008D919C91AE014F5F5F4F0B2D0E946802D8
:105E30006C010981E02FF0E0FF87EE8700FF05C0CD
:105E4000FE85F3FD02C01DE209C0F1FE02C01BE2A7
:105E500005C0F2FC02C010E001C010E28E859F85F3
:105E60008C709070892B09F444C0112311F483E0E5
:105E700001C084E0881510F088240EC0881AF3FC55
:105E80000BC0D301ED91FC910190F081E02DC10197
:105E900060E209958A94A9F7112349F0D301ED91A5
:105EA000FC910190F081E02DC101612F0995BE8523
:105EB000B3FF03C00AE513E012C00EE513E00FC004
:105EC000E114F10409F06052D301ED91FC910190CD
:105ED000F081E02DC10109950F5F1F4F05C0EF2C28
:105EE000FF24B0E1EB22FF24F8016491662341F71F
:105EF00048C1F7FE13C0BC0CFE85F4FF04C08A81C4
:105F0000813309F4BA941B141CF0BB24B3942DC044
:105F100048E04B1550F538E0B32E27C0F6FC25C0FD
:105F2000892D90E08C159D054CF05CEFC5165FEF58
:105F3000D50624F080E8F82A01C09A94992049F007
:105F4000E2E0F0E0EC0FFD1FE90DF11D80818033F0
:105F5000A1F3F7FE0AC0B92CB394892D90E0C816BE
:105F6000D90614F0992401C09C18F7FC03C025E061
:105F700030E009C01C141D041CF021E030E003C017
:105F800096012F5F3F4F112311F02F5F3F4F992054
:105F900029F0892D90E00196280F391F882D90E077
:105FA0002817390714F0882401C0821A4F2C552471
:105FB000C20189709070892B59F00CC0D301ED910A
:105FC000FC910190F081E02DC10160E209958A9475
:105FD0008820A1F7112349F0D301ED91FC910190A4
:105FE000F081E02DC101612F099543FE0BC00CC06B
:105FF000D301ED91FC910190F081E02DC10160E3AE
:1060000009958A948820A1F7F7FE51C08601D7FE32
:1060100002C000E010E076010894E11CF11CE01AD7
:10602000F10AE1E0F0E0EC0FFD1FEE0EFF1E26018D
:106030004B185108892D90E0AA24BB24A81AB90A4C
:10604000FFEF0F3F1F0749F4D301ED91FC91019041
:10605000F081E02DC1016EE20995C016D10634F041
:10606000401651061CF4F701608101C060E3015045
:1060700010400894E11CF11C0A151B054CF0D301DB
:10608000ED91FC910190F081E02DC1010995D8CFEF
:106090000C151D0541F48A81863320F4853319F4EB
:1060A000BE85B4FF61E3D301ED91FC9165C06A81C7
:1060B000613309F00F7ED301ED91FC910190F081E5
:1060C000E02DC10109959920E1F0D301ED91FC91FA
:1060D0000190F081E02DC1016EE2099512E0E1E04E
:1060E000F0E0EC0FFD1FE10FF11D60811F5FD30198
:1060F000ED91FC910190F081E02DC10109959A94F8
:1061000071F7D301ED91FC910190F081E02D44FCF9
:1061100002C065E601C065E4C1010995D7FC05C070
:10612000C114D10441F404FF06C0D094C194D10835
:10613000D3946DE201C06BE2D301ED91FC9101902B
:10614000F081E02DC101099560E305C06F5FE6EFC6
:10615000FFEFCE0EDF1EFAE0CF16D104BCF7D3015D
:10616000ED91FC910190F081E02DC1010995D301E1
:10617000ED91FC916C2D605D0190F081E02DC101ED
:106180000995CC84DD8478C1933631F0933799F04A
:10619000933509F061C023C0F601808189835E01D7
:1061A0000894A11CB11C42E050E0C40ED51E21E0B1
:1061B000E22EF12C12C0D601AD90BC9016FD03C0AA
:1061C0006FEF7FEF02C0692D70E0E2E0F0E0CE0EED
:1061D000DF1EC5010E944D047C011F7713C0D6014C
:1061E000AD90BC9016FD03C06FEF7FEF02C0692D2C
:1061F00070E0E2E0F0E0CE0EDF1EC5010E94420436
:106200007C01106813FF0BC023C0D301ED91FC91FA
:106210000190F081E02DC10160E209958A94882DFA
:1062200090E0E816F90688F313C0F50117FD6591B3
:1062300017FF61915F01D301ED91FC910190F08115
:10624000E02DC101099581108A940894E108F108B4
:10625000E114F10451F710C1943611F0993699F513
:1062600017FF0AC0F601208131814281538184E009
:1062700090E0C80ED91E0CC0D6018D919C919C0156
:10628000442737FD4095542FE2E0F0E0CE0EDF1EAC
:106290009FE6F92EF12257FF09C0509540953095A1
:1062A00021953F4F4F4F5F4FF0E8FF2ACA01B901D8
:1062B000AE014F5F5F4F2AE030E00E940A02E82EF5
:1062C0004B89E41A41C0953721F41F7E2AE030E063
:1062D0001CC0197F9F3661F0903720F4983509F083
:1062E000CEC00FC0903739F0983709F0C8C004C04D
:1062F00028E030E00AC0106114FD146020E130E0B5
:1063000004C014FD166020E132E017FF08C0D6017A
:106310006D917D918D919C91E4E0F0E008C0D601F3
:106320008D919C91BC0180E090E0E2E0F0E0CE0E27
:10633000DF1EAE014F5F5F4F0E940A02E82EFB890D
:10634000EF1A8FE7F82EF122F6FE0BC04EEFF42283
:10635000E91438F4F4FE07C0F2FC05C05FEEF52244
:1063600002C01E2D01C0192DF4FE0DC0FE01EE0D60
:10637000F11D8081803319F489EEF82208C01F5F77
:10638000F2FE05C003C08F2D867809F01F5F0F2D28
:10639000F3FC18C0F0FE13C0181510F09E2C0FC0AF
:1063A0009E2C980C911A182D0AC0D301ED91FC91E6
:1063B0000190F081E02DC10160E209951F5F181581
:1063C000A0F304C0181510F4811A01C0882404FF3A
:1063D00017C0D301ED91FC910190F081E02DC10136
:1063E00060E3099502FF29C0D301ED91FC91019072
:1063F000F081E02D01FD02C068E712C068E510C021
:10640000802F8678D1F001FF02C06BE201C060E20C
:10641000F7FC6DE2D301ED91FC910190F081E02D4C
:10642000C10109950AC0D301ED91FC910190F08161
:10643000E02DC10160E309959A94E914A0F3EA9470
:10644000D301ED91FC91A1E0B0E0AC0FBD1FAE0D0A
:10645000B11D0190F081E02DC1016C910995EE20F4
:1064600071F70AC0D301ED91FC910190F081E02D0C
:10647000C10160E209958A948820A1F71DCC649639
:106480000FB6F894DEBF0FBECDBFCF91DF911F9145
:106490000F91FF90EF90DF90CF90BF90AF909F90C3
:1064A0008F907F906F905F904F903F902F900895C6
:1064B000F999FECF72BD61BDF89A80B50895F9993A
:1064C000FECF1FBA72BD61BD40BD0FB6F894FA9AF7
:1064D000F99A0FBE08950F93FC016115710511F42F
:1064E00080E011C0218332834383548372876187A4
:1064F0000170000F000F000F8081877F802B82606A
:106500008B7F808381E00F910895CF93DF93EC011F
:106510000E9440339B01AC018D819E81AF81B88583
:10652000281739074A075B0728F4888184FD02C0D1
:1065300060E00DC089819A81AB81BC81820F931F7D
:10654000A41FB51F8D839E83AF83B88761E0222788
:1065500057FD2395332744275527922F9170929505
:10656000907F88818F7E892B8883862FDF91CF91C2
:106570000895CF93DF93EC01888182FF0FC0CE0195
:106580000E948532882351F0E985FA85309709F019
:106590000995888183FF02C08B7F8883DF91CF912B
:1065A0000895CF93DF93EC0189859A85892BE1F0DB
:1065B00089819A81AB81BC810097A105B105A1F0C9
:1065C0000E94403329813A814B815C81260F371F1D
:1065D000481F591F2D833E834F83588788818460CD
:1065E0008F7E888381E001C080E0DF91CF910895A4
:1065F0001F920F920FB60F9211242F933F938F93F8
:106600009F93AF93BF938091960690919706A09128
:106610009806B091990630919A060196A11DB11D78
:10662000232F2D5F2D3720F02D570196A11DB11D71
:1066300020939A068093960690939706A0939806C7
:10664000B09399068091920690919306A09194063A
:10665000B09195060196A11DB11D8093920690936D
:106660009306A0939406B0939506BF91AF919F9126
:106670008F913F912F910F900FBE0F901F90189503
:106680008FB7F8942091960630919706409198061E
:10669000509199068FBFB901CA0108959B01AC01C1
:1066A0007FB7F8948091920690919306A0919406FA
:1066B000B091950666B5A89B05C06F3F19F001968D
:1066C000A11DB11D7FBFBA2FA92F982F8827860F34
:1066D000911DA11DB11D62E0880F991FAA1FBB1F4C
:1066E0006A95D1F7BC012DC0FFB7F894809192064E
:1066F00090919306A0919406B0919506E6B5A89B5B
:1067000005C0EF3F19F00196A11DB11DFFBFBA2FC3
:10671000A92F982F88278E0F911DA11DB11DE2E092
:10672000880F991FAA1FBB1FEA95D1F7861B970BED
:10673000885E9340C8F2215030404040504068513C
:106740007C4F211531054105510571F608950197DA
:1067500039F0880F991F880F991F02970197F1F759
:106760000895789484B5826084BD84B5816084BDC9
:1067700085B5826085BD85B5816085BDEEE6F0E0BA
:10678000808181608083E1E8F0E010828081826016
:106790008083808181608083E0E8F0E08081816097
:1067A0008083E1EBF0E0808184608083E0EBF0E0C7
:1067B000808181608083EAE7F0E08081846080836B
:1067C0008081826080838081816080838081806815
:1067D00080831092C10008951F920F920FB60F92FE
:1067E00011242F933F934F935F936F937F938F93D6
:1067F0009F93AF93BF93EF93FF9380919B069091EC
:106800009C06892B29F0E0919B06F0919C06099546
:10681000FF91EF91BF91AF919F918F917F916F9178
:106820005F914F913F912F910F900FBE0F901F904E
:1068300018951F920F920FB60F9211242F933F932A
:106840004F935F936F937F938F939F93AF93BF9378
:10685000EF93FF9380919D0690919E06892B29F0DE
:10686000E0919D06F0919E060995FF91EF91BF91F1
:10687000AF919F918F917F916F915F914F913F91D8
:106880002F910F900FBE0F901F901895CF93DF930D
:10689000482F50E0CA018C569C4FFC01349140585F
:1068A0005C4FFA018491882369F190E0880F991F69
:1068B000FC01EE59FC4FA591B491FC01E459FC4F49
:1068C000C591D491662351F42FB7F8948C91932FEE
:1068D000909589238C93888189230BC0623061F461
:1068E0002FB7F8948C91932F909589238C9388815E
:1068F000832B88832FBF06C09FB7F8948C91832B7E
:106900008C939FBFDF91CF910895482F50E0CA012B
:1069100088559C4FFC012491CA018C569C4FFC0168
:10692000949140585C4FFA013491332309F440C0EC
:10693000222351F1233071F0243028F42130A1F0CA
:10694000223011F514C02630B1F02730C1F02430C8
:10695000D9F404C0809180008F7703C080918000BB
:106960008F7D8093800010C084B58F7702C084B57E
:106970008F7D84BD09C08091B0008F7703C0809166
:10698000B0008F7D8093B000E32FF0E0EE0FFF1F8B
:10699000E459FC4FA591B4912FB7F894662321F4E4
:1069A0008C919095892302C08C91892B8C932FBF59
:1069B00008958093A0020895982F8E3008F09E507D
:1069C00097708091A0028295880F880F807C892B18
:1069D00080937C0080917A00806480937A0080911B
:1069E0007A0086FDFCCF2091780040917900942FA9
:1069F00080E030E0282B392BC9010895CF92DF9237
:106A0000EF92FF920F931F93CF93DF937C016B0163
:106A10008A01C0E0D0E00FC0D6016D916D01D701B1
:106A2000ED91FC910190F081E02DC7010995C80F0F
:106A3000D91F015010400115110571F7CE01DF91EA
:106A4000CF911F910F91FF90EF90DF90CF9008951D
:106A5000CF93DF930E94B1330E945529C0E0D0E06C
:106A60000E94872B2097E1F30E940000F9CF505835
:106A7000BB27AA270ED041C201D230F006D220F0A7
:106A800031F49F3F11F41EF4C0C10EF4E095E7FB12
:106A9000B6C1E92F54D280F3BA176207730784078F
:106AA000950718F071F49EF56CC20EF4E0950B2E6C
:106AB000BA2FA02D0B01B90190010C01CA01A00150
:106AC0001124FF27591B99F0593F50F4503E68F1AB
:106AD0001A16F040A22F232F342F4427585FF3CFEC
:106AE000469537952795A795F0405395C9F77EF4BD
:106AF0001F16BA0B620B730B840BBAF09150A1F006
:106B0000FF0FBB1F661F771F881FC2F70EC0BA0F8B
:106B1000621F731F841F48F4879577956795B79513
:106B2000F7959E3F08F0B3CF9395880F08F099270B
:106B3000EE0F979587950895A1D158F080E891E0E0
:106B400009F49EEFA2D128F040E851E059F45EEF3D
:106B500009C05BC116C2E92FE078F1D168F3092EB4
:106B6000052AC1F3261737074807590738F00E2EB4
:106B700007F8E02569F0E025E0640AC0EF6307F854
:106B8000009407FADB01B9019D01DC01CA01AD01E6
:106B9000EF934AD0B2D10AD05F91552331F02BED5B
:106BA0003FE049E450FD49EC63CF0895DF93DD27D2
:106BB000B92FBF7740E85FE31616170648075B0753
:106BC00010F4D92FE9D19F938F937F936F93BCD209
:106BD000E8E6F0E01DD191D12F913F914F915F9167
:106BE000EED1DD2349F09058A2EA2AED3FE049ECCE
:106BF0005FE3D0785D274DDFDF917FC1DCD008F403
:106C000081E008954AD1E39589C10CD076C13DD188
:106C100040F034D130F021F45F3F19F0F0C0511151
:106C2000B1C1F3C08CD198F39923C9F35523B1F3C3
:106C3000951B550BBB27AA2762177307840738F0EB
:106C40009F5F5F4F220F331F441FAA1FA9F333D04A
:106C50000E2E3AF0E0E830D091505040E695001CFE
:106C6000CAF729D0FE2F27D0660F771F881FBB1FBA
:106C7000261737074807AB07B0E809F0BB0B802D94
:106C8000BF01FF2793585F4F2AF09E3F510568F0E0
:106C9000B6C078C15F3FECF3983EDCF386957795FC
:106CA0006795B795F7959F5FC9F7880F911D9695E2
:106CB000879597F90895E1E0660F771F881FBB1F3E
:106CC000621773078407BA0720F0621B730B840BEB
:106CD000BA0BEE1F88F7E095089504D06894B111BF
:106CE00051C1089534D188F09F5790F0B92F99275A
:106CF000B751A0F0D1F0660F771F881F991F1AF0C7
:106D0000BA95C9F712C0B13081F03BD1B1E0089516
:106D100038C1672F782F8827B85F39F0B93FCCF397
:106D2000869577956795B395D9F73EF490958095BC
:106D3000709561957F4F8F4F9F4F0895E89409C0DC
:106D400097FB3EF490958095709561957F4F8F4F9E
:106D50009F4F9923A9F0F92F96E9BB279395F695B4
:106D6000879577956795B795F111F8CFFAF4BB0F32
:106D700011F460FF1BC06F5F7F4F8F4F9F4F16C096
:106D8000882311F096E911C0772321F09EE8872F20
:106D9000762F05C0662371F096E8862F70E060E0DC
:106DA0002AF09A95660F771F881FDAF7880F969555
:106DB000879597F90895990F0008550FAA0BE0E8F9
:106DC000FEEF16161706E807F907C0F012161306AD
:106DD000E407F50798F0621B730B840B950B39F4ED
:106DE0000A2661F0232B242B252B21F408950A2653
:106DF00009F4A140A6958FEF811D811D089597F993
:106E00009F6780E870E060E008959FEF80EC089550
:106E1000DF93CF931F930F93FF92EF92DF927B014B
:106E20008C01689405C0DA2EEF01C9D0FE01E89408
:106E3000A5912591359145915591AEF3EF0129DE4C
:106E4000FE019701A801DA9479F7DF90EF90FF90A7
:106E50000F911F91CF91DF9108959F938F937F930F
:106E60006F93FF93EF939B01AC019DD0EF91FF9146
:106E7000CFDF2F913F914F915F9195C000240A94ED
:106E80001616170618060906089500240A94121605
:106E90001306140605060895B8CF59D0E8F3E89410
:106EA000EFEFBB273FE048EC5FE76B3D73078407DC
:106EB000950708F1FF279F57B25A6A4D7F40894CCA
:106EC000F04032F4BE556542704F8643FF4F089440
:106ED000EE1F915030F0BB0F661F771F881FFF1FFA
:106EE000EBCF9EE7882332F0BB0F661F771F881F0A
:106EF0009A95C1F79395E09565C1092E0394000C0E
:106F000011F4882352F0BB0F40F4BF2B11F460FF43
:106F100004C06F5F7F4F8F4F9F4F0895EF93E0FF47
:106F200006C0A2EA2AED3FE049EC5FEBB2DDE5DF07
:106F30000F90039401FC9058E5E9F0E08ECF57FDE7
:106F40009058440F551F59F05F3F71F04795880FD7
:106F500097FB991F61F09F3F79F08795089512166E
:106F600013061406551FF2CF4695F1DF08C016161A
:106F700017061806991FF1CF8695710561050894CB
:106F80000895E894BB2766277727CB0197F90895E2
:106F900012DF08F48FEF08959B01AC0160E070E010
:106FA00080E89FE332CE0BD0A8CF68DF28F06DDFFA
:106FB00018F0952309F023CF28CF1124E3CFBFDFAA
:106FC000A0F3959FD1F3950F50E0551F629FF001FC
:106FD000729FBB27F00DB11D639FAA27F00DB11D55
:106FE000AA1F649F6627B00DA11D661F829F2227DE
:106FF000B00DA11D621F739FB00DA11D621F839F65
:10700000A00D611D221F749F3327A00D611D231F3A
:10701000849F600D211D822F762F6A2F11249F5788
:1070200050408AF0E1F088234AF0EE0FFF1FBB1FAB
:10703000661F771F881F91505040A9F79E3F51054A
:1070400070F0DDCE9FCF5F3FECF3983EDCF386958A
:1070500077956795B795F795E7959F5FC1F7FE2BF5
:10706000880F911D9695879597F9089570DFE0F048
:107070009E37D8F09639B8F49E3848F4672F782FA9
:107080008827985FF9CF8695779567959395953979
:10709000D0F3B62FB1706B0F711D811D20F4879551
:1070A00077956795939573C08DC06CCF11F40EF4EE
:1070B000ACCE88C04CDFD0F39923D9F3CEF39F57E1
:1070C000550B87FF8FD056959795B0E020F4660F4B
:1070D000771F881FBB1F1F930F9300249001A001EF
:1070E0008001F001A0E80E0F1F1F0A1E511D601B3A
:1070F000710B8009B50B48F4600F711F801DB51F1F
:107100000E1B1F0B0A0A510907C02E0F3F1F4A1FF3
:107110000E0F1F1F0A1E511D660F771F881FBB1FF2
:10712000A695F795E795F8F60617170708065B0783
:10713000211D311D411D0F911F91B901842F9158BF
:10714000880F9695879508959B01AC012CCFDF930E
:10715000D92FA3DEE695D7952AED3FE049E45FE31A
:10716000B33A6207730784079507D7952AF0A2EA16
:1071700049EC90688EDCC1DEE3EBF0E06EDEDD0F03
:107180000BF00ADFDD0F0BF49058DF910895882390
:1071900071F4772321F09850872B762F07C0662350
:1071A00011F499270DC09051862B70E060E02AF011
:1071B0009A95660F771F881FDAF7880F969587953F
:1071C00097F908959F3F49F0915028F48695779557
:1071D0006795B7959F5F80389F4F880F96958795E5
:1071E00097F9089591505040660F771F881FD2F786
:1071F000089597FB092E07260AD077FD04D049D0C1
:1072000006D000201AF4709561957F4F0895F6F727
:10721000909581959F4F0895A1E21A2EAA1BBB1B42
:10722000FD010DC0AA1FBB1FEE1FFF1FA217B30752
:10723000E407F50720F0A21BB30BE40BF50B661F68
:10724000771F881F991F1A9469F76095709580952C
:1072500090959B01AC01BD01CF01089597FB092ECC
:1072600005260ED057FD04D0D7DF0AD0001C38F415
:1072700050954095309521953F4F4F4F5F4F089562
:10728000F6F790958095709561957F4F8F4F9F4F42
:107290000895AA1BBB1B51E107C0AA1FBB1FA6175D
:1072A000B70710F0A61BB70B881F991F5A95A9F7AF
:1072B00080959095BC01CD010895EE0FFF1F0590BC
:0A72C000F491E02D0994F894FFCF3B
:1072CA002563002563256300256325326925632527
:1072DA00303269006E6F2074656D70002563253148
:1072EA002E356625630025632535692563002563E8
:1072FA0025352E32662563006D616E007374310088
:10730A007374320073743300737434007374350009
:10731A007374360070682000636C20007672200057
:10732A00686C200061702000727462006C616E00EB
:10733A0070702000706F6900616320000061742022
:10734A00002563257300256325332E3069256300E4
:10735A002534692563256300256325336925630080
:10736A0025737C2563257325630020C0C0C0C0C077
:10737A00C7C0C0C0C0C0200025342E3066256300B7
:10738A00256325332E3066256300256325352E3087
:10739A006625630025632531312E36667C256325F3
:1073AA0031312E36660025632532690025332E31A8
:1073BA00662563007C7C766F6C7420646976207223
:1073CA006174696F3A2020253569007C7C616D7093
:1073DA00206F66667365743A2020202020202535A8
:1073EA0069007C7C616D702070657220766F6C74A8
:1073FA003A20202020253569002020202020202026
:10740A00202020202000202064697361726D656449
:10741A00202000206E6F2074656C20636F6D200041
:10742A00206E6F20677073206669782000202062C2
:10743A00617474206C6F772020006C696E6B207108
:10744A0075616C697479002573002000A306000039
:10745A00E803E803E803E8039DFF0164AE4721411E
:10746A000100000000A005FE349E04A104A404A7A4
:10747A0004932B00070E091C1B1215383F363124C2
:10748A00232A2D70777E796C6B6265484F4641548A
:10749A00535A5DE0E7EEE9FCFBF2F5D8DFD6D1C43A
:1074AA00C3CACD90979E998C8B8285A8AFA6A1B4AA
:1074BA00B3BABDC7C0C9CEDBDCD5D2FFF8F1F6E35B
:1074CA00E4EDEAB7B0B9BEABACA5A28F88818693CA
:1074DA00949D9A2720292E3B3C35321F18111603FA
:1074EA00040D0A5750595E4B4C45426F68616673EA
:1074FA00747D7A898E878095929B9CB1B6BFB8AD10
:10750A00AAA3A4F9FEF7F0E5E2EBECC1C6CFC8DD09
:10751A00DAD3D4696E676075727B7C51565F584DB9
:10752A004A4344191E171005020B0C21262F283D29
:10753A003A33344E49404752555C5B7671787F6ADC
:10754A006D64633E39303722252C2B0601080F1A49
:10755A001D1413AEA9A0A7B2B5BCBB9691989F8A79
:10756A008D8483DED9D0D7C2C5CCCBE6E1E8EFFA69
:10757A00FDF4F3C2C0C0C1C0C0C1C0C0C4C0C0C154
:10758A00C0C0C1C0C0C3C0C0C1C0C0C1C0C0C5C0E6
:10759A00C0C1C0C0C1C0C000000000A92CFE341A7E
:1075AA002C4A2C7A2C972C302CB82BFE2C6E2D00C2
:00000001FF
